:020000040800F2
:10000000401C0020BD620008D9620008DD620008C3
:10001000E1620008E5620008E962000800000000F3
:10002000000000000000000000000000ED62000879
:10003000F162000800000000F5620008655A00083F
:10004000FD620008016300080563000809630008F9
:100050000D630008116300081563000819630008A8
:100060001D63000821630008256300082963000858
:100070002D63000831630008356300083963000808
:100080003D6300084163000845630008000000006C
:1000900000000000000000000000000049630008AC
:1000A0004D63000851630008556300085963000858
:1000B0005D6300086101000865630008696300086A
:1000C0006D63000871630008756300081F1F000856
:1000D0007D630008175900088563000889630008DC
:1000E0008D6300089163000895630008000000001C
:1000F0000000000000000000000000000000000000
:1001000000000000000000000000000000000000EF
:100110000000000000000000996300089D630008D3
:10012000012100F01F029140DFF8002E400942F843
:10013000201070470901002807D5DFF8D42B00F004
:100140000F00801800F8041C7047DFF8042E81545B
:10015000704780B501F092F801D31046194604BDEE
:1001600038B5DFF8B04B2088C0071FD5DFF8E85D51
:100170002878002811D100F073FA286F012804DBD9
:10018000002180B201F0E0F804E00021404280B29A
:1001900001F0DAF80120287003E000F0EAFB00200B
:1001A000287020884FF6FE71084020802088800744
:1001B00004D520884FF6FD710840208031BD2DE91F
:1001C000F04F83B0DFF83C0CB0F91A70DFF8386CF0
:1001D0000024DFF8385C0246D2E9040122462B46AF
:1001E00001F0E6F880468946781007EB90708010A1
:1001F00001F0BEF942464B4601F0DAF82246DFF83C
:10020000103C01F0CDF9C6E91801DFF8080CB0F98F
:100210001A700246D2E9040122462B4601F0C8F8C2
:1002200004460D46781007EB9070801001F0A0F99D
:1002300022462B4601F0BCF80022DFF8D43B01F047
:10024000AFF9DFF8142DC2E91A014FF4B474DFF8E6
:10025000B40BB0F918006043182190FBF1F001F0E5
:1002600087F982468B46DFF8B07BC7E900ABDFF841
:10027000A40BB0F918006043182190FBF1F001F0D5
:1002800077F980468946C7E90289DFF8782BD2E9F9
:100290000201C7E90401DFF87C4BD4E90223C7E976
:1002A0000623D6E9044522462B4601F081F801F0E9
:1002B000A7FA3067D7E9060122462B4601F078F805
:1002C00001F09EFAB067306F01F052F902460B461A
:1002D0005046594601F064F9C6E91401B06F01F0C7
:1002E00047F902460B464046494601F059F9DFF806
:1002F000682CC2E916010020DFF8341C22462B4688
:1003000001F056F802460B460020DFF8481C01F0C9
:1003100047F9CDE900014FF00008C14644464D467B
:10032000274614E0D6E9140122462B4601F092FA42
:1003300004460D46DDE9000122462B4601F038F85F
:1003400052465B4601F086FAC6E906017F1CD6E9F3
:1003500006AB306F8742E5DB44464FF080452246CE
:100360002B465046594601F023F8C6E906012746B8
:1003700018E040464946DFF8E0CBDCE9162301F0FF
:1003800069FA80468946DDE9000142464B4601F0A4
:100390000FF852465B4601F05DFADFF8BC2BC2E96C
:1003A00006017F1CDFF8B00BD0E906ABB06F8742C7
:1003B000DFDB22462B465046594600F0F9FFDFF8B6
:1003C000982BC2E90601306F401E3067B06F401EA7
:1003D000B067DFF8885BDFF82C2AD2E908012246F3
:1003E0002B4600F0E5FF4FF06632DFF8743B01F07A
:1003F000D7F802460B462046DFF8581BFFF7A9FE48
:100400002246DFF8603B00F0D3FF01F097FAB066B8
:10041000DFF8002AD2E9080122462B4600F0C8FF87
:100420004FF06632DFF8383B01F0BAF802460B466F
:100430002046DFF8201BFFF78CFE2246DFF8583CF1
:1004400000F0B6FF01F07AFADFF80C1B4867BDE850
:10045000F78F2DE9FF47DFF8444CDFF8445C0026B6
:100460003746B2462DE02046294601F093FA8046F1
:1004700089460020DFF82C1C22462B4600F098FF0E
:1004800001F088FADFF8202CDFF8203C00F090FF24
:1004900042464B4601F0DEF902460B4630463946ED
:1004A00000F0ECFE01D216461F46DFF8F00BDFF835
:1004B000001C22462B4601F0CDF904460D460AF1F8
:1004C000010ABAF5806FCEDBDFF8E80BDFF8E81B36
:1004D00032463B4601F064F8CDE902014FF0000AD4
:1004E0005646DFF8D87B58E02046294601F052FAFC
:1004F000CDE900013046DFF8AC1B22462B4600F068
:1005000057FF8046894601F045FADFF89C2BDFF85B
:100510009C3B00F04DFFDDE9002301F09BF9DDE994
:10052000022300F045FF32463B4600F041FF01F058
:1005300005FADFF88C1B21F81A002046294601F045
:100540002CFACDE900014046494601F026FADFF8D1
:10055000582BDFF8583B00F02BFF02460B46DDE935
:10056000000101F01DFADDE9022300F021FF32460F
:100570003B4600F01DFF01F0E1F9DFF88C1C21F88B
:100580001A00DFF8180BDFF8281B22462B4601F073
:1005900061F904460D460AF1010ABAF5806FA3DB42
:1005A000DFF8884C206840F002002060DFF8805CB3
:1005B000092028853046DFF87C1CDFF84C68D6E936
:1005C000042300F0EDFF01F01BF9401EA8850C206C
:1005D000A886A88940F00300A881812028800E21E8
:1005E0001D20FFF7A7FD1D20FFF79AFD206840F0B2
:1005F00000502060DFF8400C016821F440310160B8
:10060000016821F440210160DFF8301C0A6842F0E3
:1006100002020A600A6842F038020A600A6842F080
:1006200001020A60026822F440120260026822F4A9
:10063000400202600A6842F400320A600A6842F42A
:1006400060120A600A6842F480320A604021016147
:100650004FF48050DFF8E81B0860BDE8FF47AEE5C7
:100660002DE97C4FDFF8A067D6E91023DFF8D40B23
:10067000D0E90045AB4201D1A24236D0002B04D1D3
:10068000002A02D10A21C6F88010B2EB040863EBFD
:100690000509CDE90089D6E91289DDE900ABD94524
:1006A00009DC01DBD04506D2D6E91223A2186B4142
:1006B000C0E9002319E0DDE90089D6E912ABDAF1DF
:1006C000000A6BEB4B0BD9450ADC01DBD04507D2A6
:1006D000D6E91223A21A65EB0303C0E9002304E064
:1006E000C0E900230021C6F88010D0E90023D6E934
:1006F0000845A4185D41C6E90845D6F880100129CF
:100700000AD0C0F0EB80032953D029D3052900F08B
:100710000D81C0F0CC80E1E0D6E90A8918EB020235
:1007200049EB0303C6E90A23D6E90E89D6E9122369
:1007300018EB020249EB0303C6E90E23A2186B4132
:10074000C6E90823F16F491CF167D6E90C45121B75
:10075000AB41C0E90223306F8142C0F2BF8022E08A
:10076000D6E90A8918EB020249EB0303C6E90A231A
:10077000D6E90E89D6E9122318EB020249EB0303EE
:10078000C6E90E23A2186B41C6E90823F16F491C84
:10079000F167D6E90C45121BAB41C0E90223706F2B
:1007A0008142C0F29B800320C6F880000020F067E1
:1007B00094E0D6E90A8918EB020249EB0303C6E983
:1007C0000A23121BAB41CDE90023D0E90223DDE966
:1007D000000100292BDB01DC012828D399421FDC12
:1007E00001DB90421CD2D6E90E89D6E912AB18F192
:1007F000010249F1000301F093F9A0FB0A2300FB79
:100800000B3301FB0A335B0043EAD27318EB42005F
:1008100049EB03010222002301F082F9C6E90E012F
:10082000D6E90E0100292FDC2ADB2DD228E08B42ED
:100830001FDC01DB82421CD2D6E90E89D6E912AB5D
:10084000B8F1010269F1000301F06AF9A0FB0A2383
:1008500000FB0B3301FB0A335B0043EAD27318EB56
:10086000420049EB03010222002301F059F9C6E9D5
:100870000E01D6E90E01002906DB01DC012803D3B5
:100880000020C6F88000F067D6E90E01221845EB7B
:100890000103C6E90823019A002A03D000291DD1CB
:1008A00000281BD10020C6F88000F06716E0D6E9CA
:1008B0001201D6E90E23994241DC01DB90423ED27F
:1008C000D6E90E01D6E91223801A9941C6E90E0134
:1008D000D6E90E0120186941C6E90801706A810550
:1008E000890DB26EDFF8D80730F911005043831339
:1008F00000EB5340C013DFF8103933F911105143A6
:100900008A1301EB5241C913DFF8F824B2F9002031
:10091000002A00D04042DFF83029DFF830390128C2
:1009200014DB4FF400041C60106013E0D6E90E01E4
:10093000D6E912239942C3DB01DC9042C0D30020E8
:100940000146C6E90E01C6F88000C1E780241C609C
:1009500040421060DFF8E808012904DB4FF400335F
:100960000360D16003E0022303604842D060BDE829
:10097000738F2DE9F84FDFF8E045D4E91223DFF853
:10098000D058D5E90067BB4201D1B2422AD0002B32
:1009900004D1002A02D10A20C4F88000B2EB060A72
:1009A00063EB070BD4E91401594507DC01DB504523
:1009B00004D230187941C5E9000113E0D0F10008F4
:1009C00061EB4109CB4508DC01DBC24505D2301A99
:1009D00067EB0101C5E9000104E0C5E9002300203F
:1009E000C4F88000D5E90001D4E90A23161843EBC6
:1009F0000107C4E90A67D4F88020012A0AD0C0F0B0
:100A0000EB80032A51D029D3052A00F00A81C0F0D7
:100A1000CC80E1E0D4E90C2310185941C4E90C0161
:100A2000D4E91089D4E9140118EB000049EB010165
:100A3000C4E9100130187941C4E90A01E26F521C7F
:100A4000E267D4E90E67801BB941C5E90201DFF80E
:100A5000B803806F8242C0F2BF8020E0D4E90C234B
:100A600010185941C4E90C01D4E91089D4E91401E2
:100A700018EB000049EB0101C4E91001301879417D
:100A8000C4E90A01E26F521CE267D4E90E67801BD9
:100A9000B941C5E90201A06F8242C0F29D800320E6
:100AA000C4F880000020E06796E0D4E90C23101819
:100AB0005941C4E90C01801BB941C5E90401D5E9DC
:100AC000022300292EDB01DC01282BD3994222DCF2
:100AD00001DB90421FD2D4E91089D4E914AB18F19C
:100AE000010249F1000301F01BF852465B46A0FBEE
:100AF00002AB00FB03BB01FB02BB4FEA4B0B4BEA13
:100B0000DA7B18EB4A0049EB0B010222002301F0CB
:100B100007F8C4E91001D4E91001002932DC2DDB0B
:100B200030D22BE08B4222DC01DB82421FD2D4E99F
:100B30001089D4E914ABB8F1010269F1000300F0A7
:100B4000EFFF52465B46A0FB02AB00FB03BB01FB81
:100B500002BB4FEA4B0B4BEADA7B18EB4A0049EB3E
:100B60000B010222002300F0DBFFC4E91001D4E9ED
:100B70001001002906DB01DC012803D30020C4F8A2
:100B80008000E067D4E91001321847EB0103C4E9A3
:100B90000A236A69002A03D000291DD100281BD12D
:100BA0000020C4F88000E06716E0D4E91401D4E91D
:100BB000102399423EDC01DB90423BD2D4E9100184
:100BC000D4E91423801A9941C4E91001D4E9100131
:100BD00030187941C4E90A01E06A8005800D616F2F
:100BE000DFF8DC2432F910204A43931302EB53421E
:100BF000D613DFF8142632F910004843811300EBB6
:100C00005140C7138348B0F90000002800D0764255
:100C1000DFF82C06A969012913DB4FF000510160B0
:100C200012E0D4E91001D4E914239942C6DB01DCB7
:100C30009042C3D300200146C4E91001C4F88000EB
:100C4000C4E74FF400510160216F012903DB4FF02D
:100C50000041016002E04FF40041016000F086FBBA
:100C6000012E05DB0021304680B200F05BFB04E082
:100C70000021704280B200F055FBAE612767BDE8ED
:100C8000F18F10B5B44C607800280CD05E48D0F8D5
:100C90008000002807D100206070DFF8B825D2E975
:100CA000020100F039F8A07800280AD0D4F88000BA
:100CB000002806D10020A070D4E90801BDE810404A
:100CC000ACE010BD38B5504C0022E266DFF8885524
:100CD000C5E90001D5E90023D4E9180100F068FB5B
:100CE00000F0B8FFC4E9080131BD38B5DFF86C4544
:100CF000C4E90001DFF86855D4E90023D5E91A01F9
:100D000000F056FB00F0A6FFC5E90A0131BD000066
:100D100018ED00E0100400402DE9F04D04460D46AA
:100D2000DFF8E480D8F88000002815D0DFF824052B
:100D3000C0E90245012088494870D8E90E01002920
:100D400006DB01DC012803D30420C8F8800056E04C
:100D50000520C8F8800052E02A48B0F9180000F0D9
:100D600007FCDFF80025DFF8003500F021FB064620
:100D70000F4622462B4600F081FA01D234463D460A
:100D800087F000472046294632463B4600F076FA77
:100D900001D234463D460020C8F86C00C8E9004541
:100DA000D8E90423624900F003FB06460F462046BB
:100DB000294632463B4600F0F3FBDFF89824C2E9AF
:100DC0000001D8E918ABD8E9140132463B4600F0DF
:100DD000E7FB52465B4600F0EBFA00F03BFFC8E948
:100DE000120122462B465046594600F0E1FA32469F
:100DF0003B4600F0D5FB00F02DFFC8E91001BDE82F
:100E0000F08D0000E01200208810002000009042C9
:100E10000080764028130020981300202DE9F04D23
:100E200004460D46DFF83081D8F88000002813D042
:100E3000C8E90845012088F80200D8E91001002916
:100E400006DB01DC012803D30420C8F8800057E04A
:100E50000520C8F8800053E0DFF81004B0F918004E
:100E600000F086FBDFF8FC23DFF8FC3300F0A0FA8B
:100E700006460F4622462B4600F000FA01D23446C1
:100E80003D4687F000472046294632463B4600F063
:100E9000F5F901D234463D46C8E90245DFF8D003F2
:100EA000D0E904230020224900F082FA06460F46CA
:100EB0002046294632463B4600F072FBDFF8B42359
:100EC000C2E90001D8E91AABD8E9160132463B461F
:100ED00000F066FB52465B4600F06AFA00F0BAFE8C
:100EE000C8E9140122462B465046594600F060FAE4
:100EF00032463B4600F054FB00F0ACFEC8E912015C
:100F0000BDE8F08D38B5DA4CD4E9080100F0E0FE18
:100F1000D4E9182300F044FB04460D46CE48C0E94E
:100F20000045FFF7AEFE2046294634BD00E100E053
:100F30000020AC4010B5084CD4E90A0100F0C8FE0E
:100F4000D4E91A2300F02CFBC44AC2E9000110BD09
:100F500000E400E00000F03F00100020000014401A
:100F600066661A4000FEAF402DE9704F8046894604
:100F7000BF4ED6F88000002840F08C80002001464B
:100F8000C6E90E01D6E90801C6E90C0100F0A0FE91
:100F900004460D46D6E9180142464B4600F008FAD1
:100FA00022462B4600F056FC00F054FEC6E90A012A
:100FB000D6E904230020B04900F0FAF902460B46B6
:100FC000D6E9140100F0ECFA04460D46D6E906AB6A
:100FD0005046594642464B4623F0004300F04EF936
:100FE00021D20020F067404649460022134600F017
:100FF0009BFE02D2C6E9164503E085F00045C6E92E
:101000001645D6E91623D6E9180100F0D1F900F00B
:1010100021FEC6E91201D6E90001C6E9020101205C
:10102000C6F8800036E04046494621F0004152466D
:101030005B4600F0B5FA00F08FFE82468B46306FBB
:1010400000F096FA52465B4600F0B2F900F0D8FB89
:1010500070670020F067404649460022134600F0C2
:1010600063FE02D2C6E9164503E085F00045C6E9F5
:101070001645D6E91623D6E9180100F099F900F0D3
:10108000E9FDC6E91201D6E90001C6E90201022024
:10109000C6F88000BDE8708F00C6A940182D4454E2
:1010A000FB21693F00000840B81E85EB51B8BE3FE8
:1010B000FB21793F1EA7E8482EFFEF3F0000E040EC
:1010C000000000202DE9F84F80468946644ED6F88E
:1010D0008000002840F08D8000200146C6E9100104
:1010E000D6E90A01C6E90E0100F0F2FD04460D46FC
:1010F000D6E91A0142464B4600F05AF922462B46E1
:1011000000F0A8FB00F0A6FDC6E90C01584FD7E996
:1011100004230020584900F04BF902460B46D6E95B
:10112000160100F03DFA04460D46D6E906AB5046DE
:10113000594642464B4623F0004300F09FF821D227
:101140000020F067404649460022134600F0ECFDBF
:1011500002D2C6E9184503E085F00045C6E9184506
:10116000D6E91823D6E91A0100F022F900F072FD41
:10117000C6E91401D6E90201C6E904010120C6F856
:10118000800036E04046494621F0004152465B4629
:1011900000F006FA00F0E0FD82468B46B86F00F0E2
:1011A000E7F952465B4600F003F900F029FBB0670F
:1011B0000020F067404649460022134600F0B4FD87
:1011C00002D2C6E9184503E085F00045C6E9184596
:1011D000D6E91823D6E91A0100F0EAF800F03AFD42
:1011E000C6E91401D6E90201C6E904010220C6F8E5
:1011F0008000BDE8F18F1E48D0F88000401E80417D
:10120000C043C00F70470000000800201448D0F809
:101210008000401E8041C043C00F70470848012134
:1012200001604FF480410160704700001C100240D3
:1012300000040040804F324100080140007400402B
:10124000100C0140081400200874004010080140F0
:10125000D8130020F81300201814002020140020B8
:1012600000100020A245B6F3FD142E4028130020E4
:1012700088100020281400200020AC404FF4001CEF
:101280001CEB410F94BF1CEB430F09E041EA030C38
:1012900050EA4C0C52EA0C0C03D2994208BF90421F
:1012A000704714BF8B428242704750F8041B61B1F3
:1012B00050F8042BD30744BFA9F101039A18002367
:1012C000091F42F8043BFAD1EFE7704738B53148BF
:1012D000016841F004010160016841F0080101600A
:1012E0002D48016841F0007101602C4C206840F0ED
:1012F000405020602068800080082060284D2868C9
:1013000040F040702860286820F04060286000218C
:10131000012000F099FD4FF40040E060402028617A
:1013200031BD0000214A12881206FBD41D4A4FF439
:10133000004313605FF00043136000BF084340F4B4
:10134000805000F0E6BD0000184A12881206FBD457
:10135000144A4FF4004313605FF00043136000BF72
:10136000084340F4104000F0D4BD00000F4800884E
:101370000006FBD44FF400400A49086000BF0A4849
:101380005FF48001016000BF00BF00BF4021016029
:10139000704700001810024004000140040801409A
:1013A000000C014010080140100C014008300140C1
:1013B000B0B581EA030C0CF0004C40F2FF7515EA61
:1013C00011541DBF15EA1357AC42AF4239E0E4197E
:1013D00023EA455343F48013C90241F0004141EA36
:1013E000505EC7021100A7FB020200284FF0000068
:1013F000EEFB01204FF00001E3FB072118BF42F094
:101400000102401800214941E3FB0E01A4F580646C
:101410000F0302D252004041494154F101046CDDF6
:10142000470872F1004250F1000051EB0451A1F560
:1014300080115CBF41EA0C01B0BD4CEA05510020AF
:10144000B0BD05EA1357AC4214BFAF4241E050EAC9
:10145000410E1CBF52EA430E02E061460020B0BDBF
:1014600024423C441BD15FEA070EF6D0090302BFB9
:1014700001460020AEF1140EB1FA81F7AEEB07047D
:1014800001FA07FE0C37C7F1200100FA07F7C84040
:101490004EEA000E23EA455343F48013A2E733F0EB
:1014A0000043B3FA83F704BFB2FA82FE77440B3FDE
:1014B000E41BB7F1200E2FBF02FA0EF3BB40C7F1B9
:1014C000200E22FA0EFE38BF43EA0E03BA40641C17
:1014D00082E750EA410E14BF52EA430E6FF000015A
:1014E0004FF4001717EB430F8ABF194617EB410F54
:1014F000B5E74CEA05510020B0BDD4F10104B4F1C8
:1015000020070FDAC4F12007520828BF42F0010279
:1015100010FA07F501FA07F7E1BF2A43E040384324
:10152000E1400FE0352C98DCC7F1200452EA40027C
:1015300020FA07F218BF42F0010231FA07F0A14089
:101540000A43002172F1004250F1000051EB0C01FE
:10155000B0BD03681AB95A1E026008467047197870
:1015600011B94FF0FF307047591C0160187870476F
:10157000010040F10980F446404200F005F851F0C6
:1015800000416047010000BF09D0B0FA80F18840F7
:10159000C91CC1F58461090501EBD02140057047E4
:1015A0002DE9F04140F2FF7581EA030C0CF0004C8C
:1015B00015EA11541DBF15EA1357AC42AF42E9E0DA
:1015C000BC41C1F31301C3F31303801A994143F4DF
:1015D000801304D2641E4000494180185941C90259
:1015E00041EA5051B1FBF3F603FB1611A2FB06755D
:1015F000D7EBC020A94102D2761E80185941C902FA
:1016000041EA5051B1FBF3FE03FB1E11A2FB0E7524
:10161000D7EBC020A94103D2AEF1010E8018594189
:10162000890241EA9051760546EA8E2EB1FBF3F627
:1016300003FB1611A2FB0675D7EB8020A94102D24D
:10164000761E80185941C90241EA50514EEA060EF1
:10165000B1FBF3F603FB1611A2FB0675D7EBC02016
:10166000A94102D2761E80185941C90241EA50515F
:10167000B1FBF3F703FB1711A2FB0735D3EBC02037
:10168000A94167F100070CBF004247F0010766F36C
:10169000D5274FEA1E31B80814F5806414DDBD0764
:1016A00075F1004250EB0E5051EB045111F5801FC3
:1016B0005CBF41EA0C01BDE8F0814CF07F6141F074
:1016C000E0410020BDE8F081BD076D0840EA0E5002
:1016D00041F48011D4F10104B4F120060ADAC4F116
:1016E00020060200E04001FA06F3E1401843B24050
:1016F00015430EE0342C14DCC6F1200445EA400505
:101700006D0820FA06F2154321FA06F0A1400D43B8
:10171000002175F1004250F1000051EB0C01BDE8D1
:10172000F08100205FEA0C01BDE8F081CFB992188A
:101730005B41B3FA83F704BFB2FA82F6BF190B3FDD
:10174000B7F120062FBF02FA06F3BB40C7F120060F
:1017500022FA06F638BF3343BA401CB1E419641EBE
:101760002FE77F4231F00041B1FA81F404BFB0FAB3
:1017700080F6A4190B3CB4F120062FBF00FA06F145
:10178000A140C4F1200620FA06F638BF3143A0403C
:101790003C1B16E7AC421ABF05EA1357AF4214E0F0
:1017A00050EA41061CBF52EA4306BFE750EA410730
:1017B000304661461CBF41EA0551BDE8F08152EA5E
:1017C000430C08BFC143BDE8F08100204FF4001670
:1017D00016EB410F98BF16EB430F08BF16EB410FF6
:1017E00024BFC14305E016EB430F0CBF61464CEA32
:1017F0000551BDE8F0810268531C03601170704709
:1018000038B5C1F30A5440F2FF75AC4215D0002C34
:1018100004BF0B0350EA133213D000F09FFB0022E9
:10182000094B00F081FA08D8084A094BFFF726FD5A
:101830003CBFBDE8344000F081B800F0B1FB21218D
:101840000160002032BD00BF0000E0C10100C0FF08
:10185000FFFFDF41F0B44FF0004591EA030C44BFB5
:101860006B4000F0A7B800BF841A71EB030603D2E7
:10187000001BB141121973414FF4001C1CEB410FC6
:1018800034BF7CEB430443E00C0DA4EB1356352E20
:1018900050DC45EAC323DB0A45EAC121C912B6F18F
:1018A00020050DDD63FA05F6EB4086EA03051242DA
:1018B00018BF45F00105C01851F100010CD213E02A
:1018C00062FA06F5F2405540F3415A40B340F34006
:1018D0005A408018594107D349085FEA30005FEA4F
:1018E000350528BF45F0010501F58011420875F165
:1018F000004250F1000041EB0451F0BC4FF4001CD9
:101900001CEB410F38BF70470020090D09057047D7
:101910001CEB410F10D252EA43060BD0BCEB410F37
:1019200005D80C0DAB43661E342EB5DD02E0AB438B
:1019300080185941F0BC7047F0BC7047F446400D28
:1019400040EAC120490006D200F014F8004248BF26
:101950006FF00040604700F00DF84FF00041884202
:101960008CBF084640426047400D40EAC120490014
:1019700080F00D8040F00040490DA1F58061491CC8
:1019800005D4D1F11F0154BFC840C01770474FF0B4
:1019900000007047002200F009BB012200F006BBE6
:1019A000F0B44FF0004591EA030F44BF6B40FFF7DE
:1019B0005BBF00BF841A71EB030604D26E40001BAC
:1019C000B141121973414FF4001C1CEB410F34BF9D
:1019D0007CEB430684E00C0DA4EB1356362E7DDC25
:1019E000012E43DC45EAC32343EA525312BFD2021D
:1019F00092025B08240545EAC12141EA5051D2EB2D
:101A0000C020994125D407D1B0FA80F610FA06F12A
:101A100064D00020203608E0B1FA81F6B140C6F16A
:101A2000200220FA02F21143B0404FEAF474B4EB02
:101A3000465434F001064FEA74040AD8D6F500166D
:101A4000760D04F00044F04061FA06F25040F14097
:101A50004840C00A40EA415021F0004128BF5FEAF7
:101A6000500550F1000044EBD12137E045EAC32393
:101A7000DB0A45EAC121C90AB6F120050EDD42EABA
:101A80000242120CC5F1200603FA06F6EB4042EAC8
:101A900006056D42984161F100010DE062FA06F51C
:101AA000F240554063FA06FC82EA0C02F3405A40C9
:101AB0006D42904161EB030111F4801F05D1641E5A
:101AC000620502D06D004041494121F48011430874
:101AD00075F1004350F1000041EB0451F0BC704738
:101AE0001CEB410F15D223F0004352EA43060BD002
:101AF0004FEA4C0CBCEB410F04D80C0D661E342E83
:101B0000B7DDEBE7801A994150EA410608BF002192
:101B1000E4E708BF1CEB430F28BF6FF00001DDE7CF
:101B200013F0004C03D55B42524263F100039CEA80
:101B3000210C00F0178010B5644603D3494240429F
:101B400061F1000100F00EF8640004D34942404204
:101B500061F10001244203D55B42524263F100036C
:101B600010BD00001B4213D1094236D12AB1844670
:101B7000B0FBF2F002FB10C2704700F02BBCFCD3AC
:101B80000022002370470B00020000210020704754
:101B9000904271EB030CF6D370B5B1FA81F4B3FA4D
:101BA00083F52C1BA340C4F1200532FA05F633431C
:101BB000A2405FF00046E64002E05B085FEA3202C6
:101BC000841A71EB030524BF204629467641F4D3DD
:101BD00002000B003000002170BD012ACFD970B582
:101BE000140C20D0B1FA81F4B2FA82F5C4F12004C9
:101BF0006419B4F12006D6D3B2405FF00044F4403B
:101C0000002502E052085FEA3303C61A71EB020EA8
:101C100024BF3046714664416D41F3D302000B008E
:101C20002000290070BD0C46B1FBF2F102FB11450A
:101C30002D0445EA1045B5FBF2F402FB145580B2C1
:101C400040EA0545B5FBF2F002FB105240EA0440C1
:101C500070BD0000F446490006D200F011F80942B8
:101C60000DD5C8174108604700F00AF807D049426F
:101C7000404271F1000102D400205FF00041604752
:101C80004A0DA2F580621E3A0ADC5242202A18DA76
:101C9000890241F0004141EA50500021D040704794
:101CA000D2F1200210D4890241F0004141EA5051A2
:101CB000C002D04061FA02F35840D14080EA0100EE
:101CC0007047002000217047D017010070470000C6
:101CD000094240F10B80F4464942404271F1000153
:101CE00000F004F851F000416047000008BFFFF722
:101CF00049BC02460846B0FA80F150408A40C1F122
:101D00002001C8415040C91E01F58461090501EB5D
:101D1000D021400540EAD220520572F1004250F134
:101D2000000041F1000170474FF4001C1CEB410F13
:101D300094BF1CEB430F09E041EA030C50EA4C0C42
:101D400052EA0C0C03D28B4208BF8242704714BF88
:101D5000994290427047000040F2FF7C0B0D4DD03D
:101D6000634566D230B421EA035141F4801103F295
:101D7000FD3C5FEA5C0C01D300184941890041EA4F
:101D8000907180004FF440140023E202D50AB1F5AF
:101D9000100107D46D081DD2091B641900184941B0
:101DA000491BF7D56D080AD20919641B001849416F
:101DB000491BEFD56D08F7D301E0520817D0C018C2
:101DC00061419B1AAC4100184941801AA941F4D4E1
:101DD00052080AD0C01AA1419B186C410018494111
:101DE000801AA941E9D45208F4D15B1C6C41610806
:101DF0004FEA330001EB0C5130BC704750EA01034D
:101E0000FBD030B4B1FA81F311B9B0FA80F41B19E8
:101E10000B3BB3F120042FBF00FA04F19940C3F14A
:101E2000200420FA04F438BF21439840D3F1010381
:101E30009DE76345E1D011F5801FDED850EA4101EE
:101E4000DBD0D94300F0C8BA10B4394B1A6842F05D
:101E500000721A60374A0128106826D140F0090044
:101E60001060186840F0010018603348036843F4BC
:101E7000401343F4405303600368304C2340036035
:101E8000036843F4000343F400430360036823F44E
:101E900040330360036823F440230360036843F482
:101EA00000230360102303611DE040F00500106073
:101EB00023480368234C234303600368224C2340D8
:101EC00003600368214C23430360036823F04073DD
:101ED0000360036823F040630360036843F000631A
:101EE000036040230361106840F48050106018487C
:101EF000028840F6030343EAC1011143018081884F
:101F000041F044018180018841F04401018010BC0E
:101F1000704710490A889207FCD5888070470D48A1
:101F20000088C00702D50C480068004770470000D1
:101F30000400014018100240000C0140FF3F3FFF29
:101F40000008014000003030FFFF3F3F000080806C
:101F50000030014008300140F413002083B5012116
:101F600000A800F03FFA401E012811D9002100A866
:101F700000F038FA60B10198DDE90023002847BF7E
:101F80000020054900200549FFF764FCCDE9000168
:101F9000DDE9000103B000BD0000F0BF0000F03F2C
:101FA000014800F05EBA0000841000202DE9F04CDA
:101FB00004460D46164683B0DFF87803DFF8781341
:101FC00022462B46FFF7F4F98B4621F00041DFF85B
:101FD0006C23DFF86C33FFF751F9074680F0F3808C
:101FE000594600220023FFF79FFE104694BFDFF8FA
:101FF0005413DFF854133A465B46FFF72BFCFFF708
:102000009DFC070051D0FFF7B3FA0022CF4BFFF73A
:10201000CFF982468B464FF0A040CD4952465B46F1
:10202000FFF7C6F902460B4620462946FFF7B8FCE3
:1020300004460D464FF0C040C64952465B46FFF786
:10204000B7F902460B4620462946FFF7A9FC04468D
:102050000D464FF00050C04952465B46FFF7A8F9C5
:1020600002460B4620462946FFF79AFC04460D46D9
:102070000020BA4952465B46FFF79AF902460B46E2
:1020800020462946FFF78CFC04460D464FF00050D1
:10209000B34952465B46FFF78BF902460B46204692
:1020A0002946FFF77DFC04460D4607F0030086191C
:1020B000204629466FF00102AA4BFFF735FE0BD8E8
:1020C00000224FF07953FFF7D9F805D2F00740F11D
:1020D0002B810024A44D27E122462B46FFF768F907
:1020E0000746F0078B4631D5A048A1493A465B46E2
:1020F000FFF75EF99F4AA04BFFF7ACFB3A465B4601
:10210000FFF756F99D4A9E4BFFF7A4FB3A465B4604
:10211000FFF74EF99B4A9C4BFFF79CFB3A465B4608
:10212000FFF746F9994A9A4BFFF794FB3A465B460C
:10213000FFF73EF96FF05102964BFFF78BFB3A46E3
:102140005B46FFF735F90022874B37E03A465B469E
:1021500020462946FFF72CF9CDE900013A468E4882
:102160008E495B46FFF724F98D4A8E4BFFF772FBD1
:102170003A465B46FFF71CF98B4A8C4BFFF76AFB2C
:102180003A465B46FFF714F9894A8A4BFFF762FB30
:102190003A465B46FFF70CF9874A884BFFF75AFB34
:1021A0003A465B46FFF704F9854A864BFFF752FB38
:1021B000DDE90023FFF7FCF822462B46FFF74AFB38
:1021C00004460D46B0E0C5F30A5240F2FF739A424E
:1021D0000BD0002A04BF280354EA103013D1002E7C
:1021E00000F0F2800024604DEEE0280354EA103045
:1021F00040F0EA80FFF7D4FE212101604FF0FF306C
:102200006FF00041E2E0CDE9004500A800F02AF9B6
:10221000DDE900458619204629466FF00102514B41
:10222000FFF782FD0AD800224FF07953FFF726F816
:1022300004D2F00778D500244B4D75E022462B469A
:10224000FFF7B6F80746F0078B4631D547484849AF
:102250003A465B46FFF7ACF8464A474BFFF7FAFAB7
:102260003A465B46FFF7A4F8444A454BFFF7F2FABB
:102270003A465B46FFF79CF8424A434BFFF7EAFABF
:102280003A465B46FFF794F8404A414BFFF7E2FAC3
:102290003A465B46FFF78CF86FF051023D4BFFF773
:1022A000D9FA3A465B46FFF783F800222E4B37E017
:1022B0003A465B4620462946FFF77AF8CDE9000109
:1022C0003A46354835495B46FFF772F8344A354B94
:1022D000FFF7C0FA3A465B46FFF76AF8324A334BDB
:1022E000FFF7B8FA3A465B46FFF762F8304A314BDF
:1022F000FFF7B0FA3A465B46FFF75AF82E4A2F4BE3
:10230000FFF7A8FA3A465B46FFF752F82C4A2D4BE6
:10231000FFF7A0FADDE90023FFF74AF822462B4633
:10232000FFF798FA04460D46B0074DD585F00041F9
:1023300020464BE083C8C96D305FE43F0000A0FF3A
:10234000FFFFDF410000E03F0000E0BF0000303E43
:10235000FB21B941B410114026A6513E5C14D33C78
:102360009A833B3BFFFF3FBE0000F03F09260A1067
:1023700039BA213E3BA861C6F97D92BE63AC30906C
:102380009F01FA3EF6FB51166CC156BFB10255557E
:102390005555A53FFFFFDFBFB08F2FC310D8E53DD8
:1023A0008F0C73A1E1E55ABE4DADE44FE31DC73E6E
:1023B0003EE3B519A0012ABFFAF010111111813FB7
:1023C000425555555555C5BF2046294603B0BDE871
:1023D000F08C0000704700001FB5FFF7E1FD2121E0
:1023E00001601FBD4268C2F30A5240F2FF739A4275
:1023F00009D14168090304BF0068002801D1012008
:1024000070470220704743685B0004BF0368002BDD
:1024100025D040F233439A1A521A012A1FDB352A7B
:1024200006DB416801F0004141600021016013E0DA
:10243000012102F01F039940491E920607D5426808
:1024400011404A40426002681143002202E00268E3
:1024500011404A40026011B14FF0FF307047002038
:10246000704770472DE97C4C064647484749D6E9F6
:10247000004522462B46FEF79BFFCDE900010022D6
:102480000023FFF751FCDDE9002399BF00204049FC
:1024900000204049FFF7DEF9CDE90001002100A846
:1024A000FFF7A0FFDDE900230020002100F08AF8FB
:1024B0004ED03949FEF77CFF82468B464FF0A04054
:1024C000364952465B46FEF773FF02460B462046EE
:1024D0002946FFF765FA04460D464FF0C0403049E3
:1024E00052465B46FEF764FF02460B4620462946ED
:1024F000FFF756FA04460D464FF000502949524660
:102500005B46FEF755FF02460B4620462946FFF77D
:1025100047FA04460D460020234952465B46FEF723
:1025200047FF02460B4620462946FFF739FA044684
:102530000D464FF000501D4952465B46FEF738FFEE
:1025400002460B4620462946FFF72AFA04460D4666
:10255000C6E90045DDE90001154A164BFEF78EFE7F
:1025600004D3154A154BFFF7DFFB05D80022144BA7
:1025700000F038F8CDE90001DDE90001FFF7DEF9F0
:1025800000F00300BDE8768C83C8C96D305FE43F7E
:102590000000E03F0000E0BF0000303EFB21B941F9
:1025A000B410114026A6513E5C14D33C9A833B3BA9
:1025B0000000C0FFFFFFDFC10100C0FFFFFFDF41E0
:1025C0000000E04190420CD141EA030C50EA4C0C6F
:1025D00007D0994205D14FF4001C1CEB410F38BFC6
:1025E0008942704770B540F2FF7601F0004C5B0005
:1025F00006EA11545D0D1ABFB442B54278E0B3EB60
:10260000410F08BF82424BD2C3F3530343F48013FC
:10261000C1F3130141F48011641B0B3C13D9C902AF
:1026200041EA5051B1FBF3FE03FB1E11A2FB0EE683
:10263000DEEBC020B14101D28018594150EA0106B9
:1026400053D00B3CEBD80B34C4F12006A14020FA48
:1026500006F6A0403143B1FBF3FE03FB1E11A2FBC3
:102660000EE6B0EB0E00B14101D28018594102BF15
:102670000146203D0020C1B3B1FA81F39940C3F176
:10268000200220FA02F211439840ED1A0A3509DBC4
:10269000C00A40EA41504CEAD12101EB055170BD1E
:1026A00023D070BDD5F10B05B5F120020DDAC5F1CF
:1026B00020020300E84001FA02F6E940934073F17A
:1026C0000043704151EB0C0170BD402D0DDC4308FF
:1026D00021FA02F0C2F1200511FA05F6334373F135
:1026E000004370415CF1000170BD6146002070BD87
:1026F00053EA020E1ABFB442B54237E0B3EB410FC2
:1027000008BF8242CCD25B08B3FA83F504BFB2FAA9
:1027100082F6AD190B3DB5F1200624BF02FA06F38F
:1027200005E0AB40C5F1200622FA06F63343AA4085
:10273000D5F1010524427FF46BAF31F00041B1FACD
:1027400081F404BFB0FA80F6A4190B3CB4F1200662
:1027500024BF00FA06F105E0A140C4F1200620FAEA
:1027600006F63143A040D4F1010455E74FF40015BB
:1027700015EB410F2CBF6FF00041EB4218BF6FF01B
:102780000041BDE87040FFF427AE70472DE9F04FDF
:10279000A1B08046002017461D4602910B900DF116
:1027A000440A6FF000490AE017F8011B0298C0477D
:1027B0000028029000F0A5820B98401C0B903878FE
:1027C00008B90B989FE22528EED1002005900690CD
:1027D0000790089009900A9001E040F0010017F876
:1027E000011F2029F9D023290DD02B2904D02D2910
:1027F00006D030290AD00CE040F0020080B2EEE7AB
:1028000040F00400FAE740F00800F7E740F010005D
:10281000F4E72A290ED12968296051F8042B296090
:10282000002A0D9204D5514240F004000D9180B26F
:102830007F1C11E000210D9109E00D99494505D05B
:1028400001EB810302EB430130390D917F1C3A7893
:10285000A2F130010A29F0D339782E2903D04FF0A4
:10286000FF310C911DE017F8011F2A2907D12968B3
:1028700029607F1C51F8042B29600C9211E0002183
:102880000C9109E00C99494505D001EB810302EB5D
:10289000430130390C917F1C3A78A2F130010A29AA
:1028A000F0D3ADF838000FF6D020397800F072FD83
:1028B00008B117F8010B8DF83A009DF83A00682826
:1028C00002BF39786829622005D06C2804BF3878A7
:1028D0006C2803D171208DF83A007F1C11A8049058
:1028E00017F8014BB4F1250023D02038022840F21C
:1028F000BB80133800F0E0800B3800F04A81401EA6
:1029000000F02381401E022840F2AE80001F00F03C
:102910001C81401F79D0401E00F0CE80401E24D084
:10292000C01E0BD0801E00F0C780C01E00F0C48007
:1029300039E125208DF8440001203DE12868286018
:1029400050F8046B286003960C9C002C04D530468C
:1029500000F02CFD044606E022460021304600F03F
:1029600041FD00B1841B069427E1296829603C24BD
:1029700051F8040B29600021CDE9000111A8039052
:10298000DDE90001049E11B908B90C9AB2B1020642
:10299000120FA0EB02123032D2B2631E3A2AA8BF45
:1029A0002732000940EA017009099A5508BF00283A
:1029B0001C4603D0039AA3199A42E8D3A0190390A6
:1029C000C4F13C010C980691814209DA401A089042
:1029D0004FF6EF71BDF838000840ADF83800ECE074
:1029E000002840F1EA809DF8380000F0140010281B
:1029F00040F0E3800D98059A801A089A801A441ACC
:102A0000012CC0F2DA800894D7E09DF83A006228E1
:102A10001AD0682806D06A280CD06C281CD07128DF
:102A200008D019E02868286050F8041B28600B982B
:102A30000880C2E02868286050F8042B28600B98B2
:102A4000C117C2E90001B8E02868286050F8041BEB
:102A500028600B980870B0E02868286050F8041BC4
:102A600028600B980860A8E02868C01D20F00702C5
:102A70002A60D2E9000108322A60CDE9000100296C
:102A800002D505982D210AE0BDF83800810702D54E
:102A900005982B2103E0C00705D50598202100F8F3
:102AA0000A10401C059011A80599081803902146AA
:102AB00000A800F0E5F980E09DF83A006C280DD000
:102AC000712818BF6A2809D12868C01D20F00702A4
:102AD0002A60D2E9000108322A6005E029682960ED
:102AE00051F8040B29600021CDE900019DF83A005E
:102AF000682803D1DDE9000180B20BE0622803D130
:102B0000DDE90001C0B205E0742818BF7A2804D1BD
:102B1000DDE900010021CDE900019DF83800000742
:102B20002ED5DDE90001002908BF002828D044F097
:102B30002000782824D10598302100F80A10401C84
:102B4000411C059100F80A401AE09DF83A00294618
:102B500000F0DCF8CDE90001002902DA05982D210A
:102B60000AE0BDF83800810702D505982B2103E063
:102B7000C00705D50598202100F80A10401C0590D3
:102B800011A8059908180390214600A800F0F5F84F
:102B900013E0012005902868286050F8041B286085
:102BA0008DF8441009E025208DF84400012005909F
:102BB0001CB18AF80140022005900D980599401A31
:102BC0000899401A0699401A0999401A0799401A1B
:102BD0000A99441A9DF83800400710D420208DF837
:102BE0004000002609E0012310AA00A9404600F099
:102BF000ABFB002840F08580761CA642F3DB059EE7
:102C00000DF1440B0AE01BF8011B0298C047002895
:102C1000029076D00B98401C0B90761E002EF2D1BD
:102C200030208DF840004FF0000B089E09E0012392
:102C300010AA00A9404600F087FB002861D10BF1E3
:102C4000010BB345F3DB069EDDF80CB00AE01BF880
:102C5000011B0298C0470028029052D00B98401CDC
:102C60000B90761E002EF2D130208DF840004FF0F0
:102C7000000B099E09E0012310AA00A9404600F0BC
:102C800063FB00283DD10BF1010BB345F3DB039847
:102C90000699079E01EB000B09E01BF8011B029847
:102CA000C047029068B30B98401C0B90761E002E14
:102CB000F3D130208DF840004FF0000B0A9E08E061
:102CC000012310AA00A9404600F03EFBC8B90BF151
:102CD000010BB345F4DB9DF8380040077FF56FAD7D
:102CE00020208DF84000002600E0761CA642BFF6AA
:102CF00066AD012310AA00A9404600F025FB00287C
:102D0000F3D04FF0FF3021B0BDE8F08F622826D01D
:102D100068281DD06A2808D06C2827D0712804D0D4
:102D2000742823D07A280CD020E00868C01D20F039
:102D300007000860D0E900230830086019461046F3
:102D400070470A680A6052F8040B0A600021704755
:102D50000A680A6052F8040B0A6000B20BE00A68C5
:102D60000A6052F8040B0A6040B204E00A680A6084
:102D700052F8040B0A60C11770472DE9FA4E054658
:102D80000A462F696F2A08BF082405D041F02000A9
:102D9000782814BF0A2410243C26D5E90001642AAF
:102DA00018BF692A81468A4605D1002903DAD9F17C
:102DB00000096AEB4A0ABAF1000F08BFB9F1000F27
:102DC0000CD1286B50B9082C36D195F83800000783
:102DD00032D530203B2687F83B002DE0E3174846EC
:102DE00051462246FEF7BEFEA4FB0023A9EB0202D9
:102DF0003032D2B2A6F1010B3A2A5E4603DB9DF8CF
:102E00000030513B9A1881465FEA010A0BF807200F
:102E100008BFB9F1000F03D0E868F1198842DDD38B
:102E2000082C09D195F83800000705D5F05D302849
:102E300002D0761E3020F055C6F13C00A861F11991
:102E4000E960296B884208DA081A28624FF6EF71A8
:102E5000288F08402887BDE8F38E00290ED595F805
:102E6000381001F01401102908D1696B6A69891AB8
:102E70002A6A891A0E1A012EA8BF2E62BDE8F38EA7
:102E80002DE9F34F8BB0D0E90089006B002801AF2A
:102E900048BF062005D404BF41F02000672802D1B6
:102EA00001200B99086340F2FF720B984168C1F34F
:102EB0000A50904220D1080302BF0B9800680028F6
:102EC0000AD10B99032088619DF8300061381A28D7
:102ED00058D30FF2B84109E00B99032088619DF89F
:102EE000300061381A284AD30FF298410B98C06815
:102EF000032200F0A3FA00E1012807DA0B9800F0A2
:102F0000D8FA012802DB00230026EDE00B9ADFF857
:102F100054B1526840F2FE3161F31E520B994A607F
:102F200040F2FE31461A4046494600220023FEF791
:102F3000A5F938BF89F0004936B247F2975070437F
:102F4000494990FBF1F636B2C6F10707012F9246C8
:102F50001BDBF80707D552465B4640464946FEF75D
:102F600027FA804689465046594652465B467F10AE
:102F7000FEF71EFA002F82468B46EAD126E00FF2BA
:102F80000041B3E70FF20041B0E77F420024374D24
:102F900012E0F80707D552465B4620462946FEF761
:102FA00007FA04460D465046594652465B46FEF720
:102FB000FFF97F1082468B46002FEAD140464946F2
:102FC00022462B46FEF7ECFA804689469DF83000F3
:102FD0000B99DFF89CB0096B40F02005662D0CBF03
:102FE00006F10A0006204718142FA8BF1327302027
:102FF0008DF804000DF10504012F3BDB40464946E6
:10300000FEF7B2FC014604F1080204234FF00A0C5B
:10301000B1FBFCFC0CEB8C04A1EB4401303102F859
:10302000011C0A21BCFBF1FE0EEB8E04ACEB440448
:1030300030345B1E714602F8024DE7D1083F012F84
:1030400002F10804D8DBFEF79DFA02460B46404623
:103050004946FEF7A5FC00225B46FEF7A9F980462B
:103060008946CBE700002440A08601000000F03F25
:1030700084D797410DF10500201A0DF1050702E0F4
:10308000401E761E7F1C39783029F9D0662D02D17A
:1030900036B2711C03E0652D0CBF012100210B9A93
:1030A000126B8B181BB29842B8BF03461BB21900B3
:1030B0001AD4814204DAC85D3528A8BF392000DA65
:1030C0003020CA19521E00E05B1E12F80159491E39
:1030D0008542F9D0392802D1C85D401CC855002965
:1030E00002D57F1E5B1C761C36B29DF830100B9803
:1030F00000961BB23A4600F003F80DB0BDE8F08F21
:103100002DE9F04305461E46D5F83080012E85B0E6
:103110008946174602DA01260FF2742749F020008B
:10312000BDF93040662808BF641C15D0672840F000
:10313000938014F1040F7CDB44457ADA95F838006B
:10314000641C000702D44645B8BFB04624B2B8EBB1
:10315000040848BF4FF0000824B2E868A969012CB0
:1031600025DA4A1C30230B54B8F1010F03DA95F825
:103170003810090702D52E211154521C18EB040FE8
:10318000B8BFC8F1000424B2A0446142B045AA61AE
:103190006962B8BF4646AB6936B2EE61324639461F
:1031A000181800F04BF9A8EB0600A862B5E0081863
:1031B000A64218DA3246394600F040F9A96971187A
:1031C000A01BB8F1010FA961686203DA95F8380015
:1031D000000705D5EA682E208854E869401CE8619C
:1031E000C5F8288099E02246394600F027F9A869F9
:1031F0002018361BB8F1010F03DA95F838100907CB
:1032000003D5EA682E218154401CA86136B2B0452E
:10321000B8BF4646E868AB6936B23246E1191818BD
:1032200000F00CF9A8693018A861A8EB06006862E4
:1032300073E0464504DA95F83810090758BFB046E0
:10324000B8F1010848BF4FF00008B9F1670F0CBF93
:103250004FF065094FF04509A969E86817F8013B87
:103260000B544A1CB8F1010F05DA95F8381009071C
:1032700058BFAA6117D52E211154531CB8F1010F64
:10328000AB6110DB761E36B2B045B8BF464636B2EB
:1032900032463946181800F0D1F8A8693018A861EC
:1032A000A8EB06006862E868A9690918200081F89F
:1032B000009003D42B2048708F1C03E02D224A700D
:1032C0008F1C644200260DF1080808E00A2200A8BD
:1032D00000F010F9019808F8010B761C009C21B24F
:1032E0000129F3DA022E06DA49F02000652804BF2E
:1032F000302007F8010B4EB9302007F8010B07E02A
:10330000761E02A8305C303007F8010B012EF7DA88
:10331000E868A9690818381AE86195F8380000F0DB
:10332000140010280DD16869A9690818696A08187D
:10333000E9690818A96A0818696B8842BCBF081AAD
:10334000286205B0BDE8F083F8B504460D46164680
:103350001F46002004E0E86A401CE8627F1E00204F
:1033600047B116F8011BA868A0470028A860F2D151
:103370004FF0FF30F2BD0000686A6C747A4C0000B8
:103380006E616E004E414E00696E6600494E460009
:10339000300000000278C9B28A421AB11CBF10F88E
:1033A000012FF9E718BF00207047000000F101036A
:1033B000810704D010F8011B89B18107FAD1026896
:1033C000B2F10131914311F0803F04BF50F8042F56
:1033D000F6E710F8011B11B110F8011BFBE7C01A4A
:1033E00070470000C9B2830706D0521E22D310F8DE
:1033F000013B9942F7D11FE0083A13D302F10402CE
:1034000041EA012141EA014150F8043B121F21BF6A
:103410004B40A3F1013C2CEA030C1CF0803FF3D09D
:10342000C9B2001F083210F8013B521E28BF91EAB2
:10343000030FF8D818BF0120401E704762B38B07F6
:1034400008D0521E11F8013B00F8013B00F0248027
:103450008B07F6D1830740F0208000BF103A07D3D6
:1034600030B4B1E83810103AA0E83810F9D230BCC6
:10347000530724BFB1E80810A0E8081044BF51F872
:10348000043B40F8043BD20724BF31F8022B20F85C
:10349000022B44BF0B7803707047083A07D3B1E89A
:1034A0000810083A40F8043B40F804CBF7D2530721
:1034B000E4E730B4436803F0004201211B031B0B17
:1034C000436004BF0368002B08D10DE00368DD0FE3
:1034D00045EA440444605B000360491E4468E3021B
:1034E000F4D523031B0B436043681A43426008462C
:1034F00030BC704791FBF2F303FB1211C0E90031BD
:103500007047000003460846C2680169521C491E04
:1035100000290161C26003D400680122002118471C
:103520004FF0FF307047034608461146C268521EEE
:1035300011F1010FC26002D00068002218477047E5
:103540002DE9F04788B0044600914FF0FF35186828
:1035500001902E460020039002920FF600370FF6DE
:10356000F4286FF0004902E00298401C0290DDF858
:1035700008A09AF80000A0F10903052B09D3202820
:1035800007D0F0B9002EB8BF0026304608B0BDE81D
:10359000F0870398401C0390012200980021A04767
:1035A000A0F109010529F4D32028F2D00399491E7E
:1035B00010F1010F0391D7D0014600980022A047D7
:1035C000D2E725280BD10AF10100029000782A28C1
:1035D00016D10298401C0290401E007811E003981A
:1035E000401C0390012200980021A0479AF8001087
:1035F0008842B9D0024600A92046FFF794FFC1E7F0
:1036000000208DF81C00002005900AE0059949452E
:1036100005D001EB810302EB430130390591401CD9
:10362000029002980278A2F130010A29EED30695A1
:1036300001784046FFF7AEFE20B10298401C029090
:10364000401E00788DF81D009DF81D00682801BF00
:1036500002990A78682A622006D06C2802BF029973
:1036600008786C2804D171208DF81D00481C029048
:10367000029801783846FFF78DFEB0B90398401CD8
:103680000390012200980021A047A0F1090105291B
:10369000F4D32028F2D00399491E10F1010F0391B1
:1036A00003D0014600980022A04700A9204600F060
:1036B00010F8012803DA002E3FF568AF65E7002E09
:1036C0009DF81E0048BF002600283FF44DAF761C31
:1036D0004AE770B505460C460020A077A068007840
:1036E000253858D01C3823D0001F022820D9133881
:1036F0001AD0C01E66D0801F1AD0801E12D0401E65
:1037000012D0401E022813D9001F0DD0401F13D025
:10371000401E012808D9001F3BD0801E04D0C01EC7
:1037200002D055E000224FE02846BDE8704034E169
:103730002846BDE8704029E2207F002835D1607F0F
:10374000622808D0682816D06A280BD06C2819D0B7
:10375000712807D016E0606850F8041B6060E068CC
:10376000087022E0606850F8042B6060E068C117C0
:10377000C2E9000119E0606850F8041B6060E0686D
:10378000088012E0606850F8041B6060E068086020
:103790000BE0012218E0E068401CE0600122206894
:1037A0000021A8470646252E01D1012070BD3246D2
:1037B00021462846FFF7B7FE16F1010F08D14FF05A
:1037C000FF3070BD4FF0FF322846BDE8704001E089
:1037D000002070BD2DE9F04F17460025002F83B063
:1037E00080460E464FF0000927D5B068401CB060F7
:1037F00000785E2806D1B068401CB060401E00789A
:10380000019000E00195B46820785D280CBF601C31
:1038100020465D21FFF7BEFD002800F0B580011BAA
:103820000091B0600098032807DB821E2D21601CE8
:10383000FFF7D8FD08B14FF001097069012804DADB
:10384000002F14BF6FF0004001203061307F60B95D
:10385000706850F804AB706007E00AF801BB012003
:10386000B077B069401EB06102253069401E3061FA
:10387000F06813D4401CF060012230680021C0477A
:1038800083461BF1010F69D0012F0CDBABF109005E
:10389000052863D3BBF1200F58D15FE0401CF060D6
:1038A0004FF0FF3B5AE0002F50D5B9F1000F0FD178
:1038B0000198009A00285946204604D1FFF792FD4E
:1038C00000284BD042E0FFF78DFD002846D13DE0B7
:1038D0000199009A0029C0B2214624D107E00B7853
:1038E0009842A4BF8B78834230DAC91CD21E032AC7
:1038F00009D34B782D2BF2D011F8013B834218BF2E
:10390000521EF4D122E04AB311F8013B834218BFA2
:10391000521EF8D11AE00B789842A4BF8B788342EC
:103920001CDAC91CD21E032A0ED34B782D2BF2D0E1
:1039300011F8013B834218BF521EF4D10EE011F87A
:10394000013B83420AD0521E002AF8D1307F002862
:103950008AD1B06900287FF480AF01255A463146EC
:103960004046FFF7E0FD0FB1022D09D0022D10D027
:10397000E80702D41BF1010F06D14FF0FF3009E038
:10398000307F30B9B06908B9002003E000208AF820
:103990000000012003B0BDE8F08F2DE9F0430C4694
:1039A000804660690128B8BF6FF00040206189B08F
:1039B0004046FFF7A7FD05462B2D18BF2D2D0DF115
:1039C000000908D18DF8005021464046FFF79AFDC6
:1039D0000DF101090546A06800780027642814BF8E
:1039E00075280A260DD0692808BF002609D06F283F
:1039F00008BF082605D070281ABF40F0200078289C
:103A00001026302D19D121464046FFF77BFD054693
:103A100045F020000127C0B278280BD1002E18BF36
:103A2000102E13D121464046FFF76CFD10260546A7
:103A300000270BE056B9082608E006BB0A261EE060
:103A4000206801220021C04705460127302D0BD1F7
:103A50002069411EE0682161401C0029E060EFD52B
:103A60004FF0FF35012700E04FB1302009F8010B7E
:103A700005E0206801220021C0470546012715F115
:103A8000010F23D0E9B26129A8BF573909DA4129CA
:103A9000A8BF373905DAA1F130020A2A34BF30391C
:103AA000FF21C9B2F0B2814210D20DF11F00814551
:103AB00038BF09F8015B2069411EE0682161401CA4
:103AC0000029E060D5D54FF0FF3501272A46214671
:103AD0004046FFF728FD47B900A881450ABF15F108
:103AE000010F00204FF0FF304DE0002089F800006A
:103AF000207F002846D1A0680078642818BF692874
:103B000007D13246002100A800F0FBFA0122A2777B
:103B10000AE03246002100A800F0A6FB0122A277AD
:103B2000A2681278702A28D0627F622A0CD0682A94
:103B300017D06A2A0ED06C2A19D0712A0AD0742A9A
:103B400018BF7A2A13D018E0626852F8043B62600A
:103B5000187017E0626852F8043B6260C3E9000124
:103B600010E0626852F8043B626018800AE0626804
:103B700052F8043B6260186004E0626852F8043B4B
:103B800062601860012009B0BDE8F0832DE9F04FB4
:103B90000C46814660690128B8BF6FF00040206183
:103BA0000025484693B0FFF7ADFC07462B2F18BF02
:103BB0002D2F0DF1080A08D18DF8087021464846CE
:103BC000FFF7A0FC0DF1090A07460026302F4FF041
:103BD0000A0818D121464846FFF794FC074647F0EB
:103BE0002000C0B2782840F0E68030200AF8010BAF
:103BF000214678200AF8010B4FF010084846FFF7DD
:103C000081FC0746D8E047F02000C0B26E285BD1A7
:103C10000AF8010B21464846FFF774FC074647F0B7
:103C20002000C0B26128A84640F0DC810AF8010BF0
:103C300021464846FFF766FC074647F02000C0B221
:103C40006E2840F0CF8121464846FFF75BFC0246D4
:103C5000282A19D021464846FFF765FC6E200AF84D
:103C6000010B00208AF80000207F002840F0ED8141
:103C7000B8F10B0F80F2C7812A46002102A800F09C
:103C8000C1FBCDE90001C9E1E1682069491C401E82
:103C900000282061E16004D4206801220021C84787
:103CA00001E04FF0FF30A0F1610107461A2921BF62
:103CB000A0F141011A2930380A28E5D35F2FE3D05B
:103CC000292F40F08F81C9E7692840F087800AF8E2
:103CD000010B21464846FFF715FC074647F0200038
:103CE000C0B26E28A84640F07D810AF8010B21463B
:103CF0004846FFF707FC074647F02000C0B2662899
:103D000040F0708121464846FFF7FCFB40F020015F
:103D1000C9B2692906D0024621464846FFF703FC8E
:103D200066209CE721464846FFF7ECFB074647F034
:103D30002000C0B26E2840F0558121464846FFF76A
:103D4000E1FB074647F02000C0B2692840F04A81F5
:103D5000E1682069491C401E00282061E16005D40B
:103D6000206801220021C847074601E04FF0FF37D5
:103D700047F02000C0B2742840F03481E168206927
:103D8000491C401E00282061E16005D42068012202
:103D90000021C847074601E04FF0FF3747F02000F9
:103DA000C0B2792840F01E81662058E720680122C1
:103DB0000021C84707460126302F0BD12069411E3C
:103DC000E0682161401C0029E060EFD54FF0FF372B
:103DD000012600E016B130200AF8010BAB4605E0E1
:103DE000206801220021C8470746012617F1010F6C
:103DF0003AD0F8B26128A8BF573809DA4128A8BFDD
:103E0000373805DAA0F130010A2934BF3038FF20F5
:103E1000C0B2404513D2BBF1240FBABF0AF8017BF0
:103E20000BF1010B6D1C2069411EE0682161401CF3
:103E30000029E060D4D54FF0FF37012614E02E2F83
:103E400012D12E200AF8010BE1682069491C401E9E
:103E500000282061E16005D4206801220021C847C4
:103E6000074601E04FF0FF37BBF1000F21D105E01D
:103E7000206801220021C84707460126302F0BD1B8
:103E800020696D1E411EE0682161401C0029E06030
:103E9000EED54FF0FF370126002D0AD530200AF865
:103EA000010B6D1C05E0206801220021C847074670
:103EB000012617F1010F24D0F8B26128A8BF5738A6
:103EC00009DA4128A8BF373805DAA0F130010A29FC
:103ED00034BF3038FF20C0B2404512D2BBF1240FAE
:103EE000BCBF0AF8017B0BF1010B2069411EE068A1
:103EF0002161401C0029E060D5D54FF0FF37012635
:103F000001E0002E6ED0B8F10A0F02BF47F0200189
:103F1000C9B2652907D0B8F10A0F63D047F0200075
:103F2000C0B270285ED10AF8017B2069401E206172
:103F300011D4E068401CE060012220680021C847DD
:103F400007462B2F18BF2D2F13D10AF8017B2069AC
:103F5000401E206105D5E068401CE0604FF0FF374F
:103F600007E0E068401CE060012220680021C847AB
:103F70000746002605E0206801220021C8470746C1
:103F80000126302F0BD12069411EE0682161401CC1
:103F90000029E060EFD54FF0FF37012600E016B1B1
:103FA00030200AF8010B4FF0000B02E04FF0FF3712
:103FB0000126A7F130000A2814D2BBF1080FBCBFBC
:103FC0000AF8017B0BF1010B2069411EE0682161B9
:103FD000401C0029E060E9D4206801220021C84784
:103FE0000746E5E73A4621464846FFF79CFA002E89
:103FF0007FF437AE02A882450ABF17F1010F0020F7
:104000004FF0FF3022E00022002102A800F0FAF970
:10401000CDE90001A90000A800F0F6F90120A07781
:1040200060680568011D607F6C2803D16160DDE96F
:10403000000104E061604C28DDE9000102D1C5E91E
:10404000000102E000F068FA2860012013B0BDE82A
:10405000F08F0000686A6C747A4C000063436E5BFA
:10406000000000002DE9F04182B080460E001D46A0
:1040700008BF00AE474600E07F1C3878A0F1090178
:104080000529F9D32028F7D02D2816BF2B2817F89B
:10409000014B2B243146384600F036F832689742FF
:1040A00008BFC6F80080326890451DD1002908BFBE
:1040B000002807D12D2C1DD1B1F1004F1CD301D800
:1040C000012819D3FDF76CFF222101600DB10120F9
:1040D00028602D2C19BF4FF0FF306FF000410020F9
:1040E0004FF00041BDE8FC812B2CE3D14FF00043A1
:1040F0009942E7D2BDE8FC81404261EB4101BDE855
:10410000FC810023AEE700002DE9F84F86B083461E
:104110000F4615460BB1002018605E4600E0761C85
:104120003078A0F109010529F9D32028F7D02D28EE
:1041300016BF2B2816F801AB4FF02B0A002D55D4D3
:10414000012D53D0252D51DA012D0ADB102D04BF8E
:104150003078302802BF707840F0200078280ED1E7
:104160000AE03078302818BF0A2508D1707840F06E
:104170002000782802D11025B61C00E008250396FF
:1041800000E0761C30783028FBD00024A046CDE932
:1041900004480FF2D800029600948DF804004FEA0C
:1041A000E57913E09DF80410401AC0B20090CDE903
:1041B000044800AAA5FB040105FB0811127809FBBD
:1041C00004110023841841EB0308761C3178A1F117
:1041D00041001A2838BF20312A460FF29000FFF71D
:1041E00001F90028DED10398B04205D10FB1C7F81C
:1041F00000B00020002134E00FF298010298695CC1
:10420000301A401A23D4012814DA00A800210078BB
:10421000201A68EB010188450CD301D8844209D3E8
:104220002A46EB17FDF79EFCDDE90423994208BFFF
:1042300090420CD0FDF7B4FE22210160069810B127
:104240000699012008604FF0FF34A04605E0BAF15E
:104250002D0F02D1644268EB480807B13E6020464A
:10426000414607B0BDE8F08F00234DE730313233CF
:104270003435363738396162636465666768696A00
:104280006B6C6D6E6F707172737475767778797A06
:104290000000000000004129211C191716151413F5
:1042A00012121111111010100F0F0F0F0E0E0E0E13
:1042B0000E0E0E0D0D0D0D0D0D0000002DE9F14D32
:1042C00087B005460C4690469A4607A800F06CF960
:1042D0008346BAF1000F1CBF0021CAF8001020F07D
:1042E0000800012834D10220009004AB079922462F
:1042F000284600F0E9F9040003D10020CDE90200CE
:104300001DE00598FDF734F9CDE90201022C16DB1A
:1043100006AE671E384DDDE9020100222B46FDF78F
:1043200047F8CDE9000156F8040BFDF721F9DDE966
:104330000023FDF78FFACDE902017F1EEBD104982F
:1043400000EB0802DDE90201534600F0DEFA42E02C
:10435000022835D1009004AB07992246284600F088
:10436000ABFB040003D10020CDE902001DE005985D
:10437000FDF7FEF8CDE90201022C16DB06AE671E42
:104380001E4DDDE9020100222B46FDF711F8CDE9B3
:10439000000156F8040BFDF7EBF8DDE90023FDF70B
:1043A00059FACDE902017F1EEBD1049902A800F071
:1043B0002BF8DDE902015346424600F0A6FA0AE076
:1043C000032802D100200E4905E0042806D14FF051
:1043D000FF306FF00041CDE9020102E00020CDE99D
:1043E00002005FEA0B70DDE9020148BF81F0004185
:1043F00008B0BDE8F08D000065CDCD410000B041B2
:104400000000F07F002359E770B504460D46606850
:10441000C0F30A5040F2FF71884207D16068000380
:1044200004BF2068002817D0022070BD20B92046A4
:10443000FFF73FF8012868DA012D0FDB40F2FF712A
:10444000091A8D420AD36068002847BF002030490E
:1044500000203049C4E90001012070BD4142A94259
:10446000616806DA6FF31E51401941EA005060603E
:1044700042E0401E63684519012205F1350062F3F0
:104480001F53352801F00041636003D361600020B1
:10449000206070BD002215F11F0F04DA226823602E
:1044A000002020356060684214D0521E2568924179
:1044B000C0F12003D2439D4045EAD272256825FA17
:1044C00000F6656805FA03F333432360636823FA53
:1044D00000F5656060680843B2F1004F606003D882
:1044E0000DD12078C0070AD52068401C20602068C4
:1044F00028B96068401C60604FF0FF3070BD606894
:10450000884204BF20680028F6D1002070BD00BF9B
:104510000000F0FF0000F07F4FEAF17CBCF1E04CBE
:104520002CBFBCF5001F11E05FEA4C0C34BFBCF19E
:104530007F5F2EE05FEA9C0C4FEA0C1C4FEA3C0CBC
:10454000C10071F100414CEB50707047C90241EA63
:104550005051C00218BF41F0010141F000414FEA43
:104560006C50C0F10900212810D240EACC7CCCF17B
:10457000200C11FA0CF070F10040CCF1200C21FA63
:104580000CF00CF0004C40EB0C0070474FEACC7084
:104590007047490011F5001F04D84FEACC10FF30D6
:1045A000C0057047C817704770B4026813460024EE
:1045B00000E05B1C1D78A5F10906052EF9D3202D1E
:1045C000F7D02D2D0CBF08242B2D00D15B1C1D789E
:1045D00045F020066E2E26D15C7844F02004612C34
:1045E00002BF9C7844F020046E2C02D013460022B7
:1045F00046E0DB1C1C4604222578282D40D114F807
:10460000015FA5F161061A2EF9D3A5F141061A2E14
:1046100024BF303D0A2DF2D325785F2DEFD0292D10
:104620002ED1631C2CE0692E2DD15D7845F020053C
:104630006E2D02BF9D7845F02005662D02D01346F1
:1046400000221DE044F0030213F8034F44F020045D
:10465000692C02BF5C7844F020046E2C10D19C7849
:1046600044F02004692C02BFDC7844F02004742C50
:1046700006D11C1D257845F02005792D08BF631C47
:10468000F1B10B601CE0302D02BF597841F02001E0
:10469000782913D1991C0A782E2A08BF491C097859
:1046A000A1F16102062A21BFA1F14102062A303997
:1046B0000A2903D29B1C44F0020201E044F00102EB
:1046C0000360104670BC70472DE9F0478CB00D4672
:1046D00014998046002001EBC1012E29A8BF2D218D
:1046E00000261E605E6001E06D1C01262F78302FD1
:1046F000FAD000270DF1000C04E01E68761C1E6045
:104700006D1C012695F800E0AEF130040A2C07D2AA
:10471000B942F2DBAEF1300607F80C607F1CEFE720
:10472000BEF12E0F08BF6D1C47B904E01E68761E4F
:104730001E606D1C01262C78302CF7D02C78A4F14B
:10474000300EBEF10A0F0CD2B94207DBA4F13006DD
:1047500000AC3E557F1C1E68761E1E606D1C012637
:10476000ECE7B94218DA00AFCF5D052F06DB00AFEA
:10477000CF1917F8014C641C07F8014C0F46196853
:10478000491C196008E000A9791811F8011C49B901
:104790001968491C19607F1E012FF4DA17B98DF8CA
:1047A00000000127002E5ED04FF0090E97FBFEFEA1
:1047B000C7F1090C0EEBCE0EE6444FF0090C9EFB40
:1047C000FCFC00210CEBCC04BEEB04040ED0012059
:1047D0000CE053F8204011F80CC004EB84040CEBFF
:1047E000440443F820400EF1010E491CB9420DDA91
:1047F00009249EFBF4F404EBC404BEEB04040DF1A5
:10480000000CE6D111F80C40401CEAE7297841F091
:104810002001652927D1294615F8017FDFF858C006
:104820002B2F16BF2D2F15F8017B2B270024A64612
:1048300009E0E64505DA0EEB8E0409EB4404A4F129
:10484000300E6D1C012495F80090A9F1300ABAF1E0
:104850000A0FEED32D2F1F6808BFCEF1000E77444C
:104860001F6004B90D461AB106B1A846C2F800800F
:104870000CB0BDE8F08700BF00E1F505455144727A
:104880006976652D6D696E69205553422033302E4F
:1048900030332E323031362032313A34343A3239F4
:1048A0000A0D00004551446D696E69203136303380
:1048B00033300A0D00000000F8B5064640F2FF71E3
:1048C0007068C0F30A50884214461D4606D001287D
:1048D00006DA3046FEF7EDFD012801DB002706E091
:1048E000726840F2FE3161F31E527260471AD6E9D7
:1048F000000122462B46FCF75BFDC6E9000139B2F8
:104900003046BDE8F440FFF77FBD2DE9FB451600BA
:1049100082B09A4600F09A80DDE90223002000214F
:10492000FDF750FE00F092800024002E4A4D43D542
:1049300076420FF23C174FF008080DE0F00707D55C
:10494000D7E9002320462946FCF732FD04460D46F0
:1049500076080837A8F10108002E18BFB8F1000F3B
:10496000ECD102A900A800F0A7F9DDE90201224676
:104970002B46FCF715FECDE90201BDF9001002A897
:10498000FFF742FD070050D5002E50D002A900A825
:1049900000F092F9DDE90201304A314BFCF708FDE5
:1049A000CDE90201BDF9001002A8FFF72DFD0700B7
:1049B0003BD5761EEAD13AE0012E36DB0FF2B00786
:1049C0004FF00808F00707D5D7E90023204629460D
:1049D000FCF7EEFC04460D4676100837012EA8F1D0
:1049E000010802DBB8F1000FECD122462B4602A8E9
:1049F000FFF762FF070018D5012E18DB02A900A8F7
:104A000000F05AF9DDE90201164A174BFCF7D0FC19
:104A1000CDE90201BDF9001002A8FFF7F5FC07007F
:104A200003D5761E012EE9DA01E03FB20FB1012F66
:104A30000CD1FDF7B5FA2221BAF1000F016005D0C3
:104A4000DAF8000040F00100CAF80000DDE90201D8
:104A500005B0BDE8F08500000000F03F436FAC6496
:104A60002806C80A3CBF737FDD4F157500000000A3
:104A70000000000000002440000000000000594039
:104A8000000000000088C3400000000084D7974168
:104A90000080E03779C34143176E05B5B5B893463A
:104AA000F5F93FE9034F384D321D30F94877825A06
:104AB0003CBF737FDD4F15752DE9F54F8BB01C465C
:104AC00016980025C0EBC008B8F1240FA8BF4FF01E
:104AD000230825600E466560002701E0761C01274B
:104AE00030783028FAD00FF2A01AA946CDF800A0ED
:104AF0000DF1040B04E02068401C2060761C0127A7
:104B0000317816225046FEF76DFC58B1C845F2DBED
:104B1000009A0FF28C11801A405C09F80B0009F121
:104B20000109EBE730782E2808BF761CB9F1000F99
:104B300008D104E02068401E2060761C01273078F0
:104B40003028F7D0317816225046FEF74BFC88B15A
:104B5000C8450CDB0FF24811A0EB0A00405C01A92C
:104B600009F8010009F101092068401E2060761C47
:104B70000127E7E7C8451ADA01A818F80000082855
:104B800006DB01A8404410F8011C491C00F8011C78
:104B9000C1462068401C206009E001A8484410F884
:104BA000010C70B92068401C2060A9F10109B9F11D
:104BB000010FF2DAB9F1000F04BF8DF804504FF085
:104BC000010920688000002F206052D0072299FB45
:104BD000F2F2C9F10701C2EBC2025118072291FBA0
:104BE000F2F20020C2EBC2028A1A05D0012503E0CE
:104BF00044F82520491C401C48450EDA072391FB48
:104C0000F3F310F80B20C3EBC303CB1A0EBF6D1CDC
:104C100054F8253002EB0312EAE7307840F0200028
:104C2000702826D1304616F8011FDFF858C02B290E
:104C300016BF2D2916F8011B2B210022002309E0A5
:104C4000634505DA03EB83020EEB4202A2F1300367
:104C5000761C012296F800E0AEF13008B8F10A0F98
:104C6000EED32D29216808BF5B425918216002B993
:104C700006460C9810B107B90B9E066028460DB089
:104C8000BDE8F08F00E1F505303132333435363789
:104C900038396162636465664142434445460000B9
:104CA000000102030405060708090A0B0C0D0E0F8C
:104CB0000A0B0C0D0E0F000038B50C460546606857
:104CC000C0F30A5040F2FF7188420BD100202880C7
:104CD0006068000304BF2068002801D0022032BDB4
:104CE000012032BD012804DA2046FEF7E2FB01284C
:104CF0000ADA626840F2FE3161F31E526260401AC5
:104D000028804FF0FF3032BD0020288032BD0000E7
:104D100030B583B0DFF8CC49A16A0978002900F0EA
:104D2000C082012101700020A16A0870DFF8B80973
:104D30000178002900F0AE8242783E2A00F08D8290
:104D4000422A00F07B82442A00F0CC80452A00F001
:104D5000DB80462A00F01781472A00F03381482A79
:104D600000F09881492A00F0D4814A2A00F00F828D
:104D70004B2A00F03B824D2A00F05582502A00F069
:104D80005D82612A10D0622A20D0632A30D0652A41
:104D900040D0662A50D0672A73D06A2A00F08380F8
:104DA000732A00F08D8075E2022940F03E828178FE
:104DB000312902D0322940F038820FF65811E06ACA
:104DC00000F03CFD00F09BFD02203EBD022940F0BA
:104DD0002C828178312902D0322940F026820FF6C8
:104DE0004811E06A00F02AFD00F089FD02203EBD76
:104DF000022940F01A828178312902D0322940F00C
:104E000014820FF63011E06A00F018FD00F077FD13
:104E100002203EBD022940F008828178312902D06B
:104E2000322940F002820FF61811E06A00F006FD08
:104E300000F065FD02203EBD022940F0F681817838
:104E400031290CD1607B0090E37B227B0FF6FC01C3
:104E5000E06A00F0F3FC00F052FD03203EBD322971
:104E600040F0E381DFF88458687B0090EB7B2A7B7D
:104E70000FF6D801E06A00F0E1FC00F040FD0420EC
:104E80003EBD022940F0D1818178312902D03229FA
:104E900040F0CB810FF6C001E06A00F0CFFC00F0DB
:104EA0002EFD02203EBD022940F0BF8181783129CC
:104EB00001D10B203EBD322940F0B78115203EBD07
:104EC000022940F0B2818178312902D0322940F0A4
:104ED000AC810FF68C01E06A00F0B0FC00F00FFD31
:104EE00002203EBD022940F0A0818178312902D004
:104EF000322940F09A810FF67401E06A00F09EFCBE
:104F000000F0FDFC02203EBD082940F08E81817832
:104F1000312919D101AADBA1801C00F06BFD019899
:104F2000000400F47F00019901F47F410818019901
:104F3000C1F3074108182060DBA1E06A00F07EFCA5
:104F400000F0DDFC0C203EBD322940F06E8101AA4C
:104F5000CCA1801C00F04EFD0198000400F47F00FD
:104F6000019901F47F4108180199C1F3074108181C
:104F7000DFF878170860CCA1E06A00F05FFC00F071
:104F8000BEFC16203EBD022940F04F8181783129B8
:104F900009D101206073C4A1E06A00F04FFC00F069
:104FA000AEFC05203EBD322940F03F810120DFF8F4
:104FB0003C174873BCA1E06A00F040FC00F09FFC85
:104FC00005203EBD042940F030818178312925D16A
:104FD00001AAC6A1801C00F00DFD0198C0B20028F6
:104FE0000AD0012811D0102809D0112810D030285B
:104FF00008D031280FD046E00020207325E10120A1
:10500000207322E1052020731FE1022020731CE1A0
:105010000320207319E10720207316E1322940F0A4
:10502000048101AAB1A1801C00F0E4FC0198C0B287
:1050300000280AD0012817D010280BD0112818D02A
:1050400030280CD0312819D01DE00020DFF89C1644
:105050000873FAE00120DFF894160873F5E00520E4
:10506000DFF888160873F0E00220DFF88016087376
:10507000EBE00320DFF874160873E6E00720DFF8A2
:105080006C160873E1E00FF2F061E06A00F0D6FB05
:1050900001203EBD082940F0C8808178312919D10E
:1050A00001AA78A1801C00F0A5FC0198000400F47E
:1050B0007F00019901F47F4108180199C1F307416C
:1050C0000818606078A1E06A00F0B8FB00F017FCF7
:1050D00002203EBD322940F0A88001AA69A1801CAF
:1050E00000F088FC0198000400F47F00019901F4AD
:1050F0007F4108180199C1F307410818DFF8EC1542
:10510000486069A1E06A00F099FB00F0F8FB02201A
:105110003EBD082940F089808178312919D101AA42
:1051200058A1801C00F066FC0198000400F47F0088
:10513000019901F47F4108180199C1F3074108184A
:10514000A06059A1E06A00F079FB00F0D8FB0220D2
:105150003EBD322969D101AA4AA1801C00F04AFC57
:105160000198000400F47F00019901F47F410818C0
:105170000199C1F307410818DFF8701588604AA14A
:10518000E06A00F05BFB00F0BAFB02203EBD0229A2
:105190004BD18178312912D10120A07342A1E06A5C
:1051A00000F04CFB00F0ABFB207B002801D0022874
:1051B00001D10E203EBD002060600D203EBD322991
:1051C00033D1DFF828550120A87337A1E06A00F039
:1051D00035FB00F094FB287B002801D0022801D188
:1051E00018203EBD2868686017203EBD02291CD1EA
:1051F0008178312909D10020A0732BA1E06A00F049
:105200001DFB00F07CFB0D203EBD32290DD100209E
:10521000DFF8D814887324A1E06A00F00FFB00F0D7
:105220006EFB17203EBD08290AD00FF2F441E06A58
:1052300000F004FB00F063FB00203EBD0329F4D125
:105240008178312901D03229EFD117A1E06A00F02D
:10525000F5FA00F054FB02203EBD8078522808D0B9
:10526000562808D0572802D076280DD0DDE7202018
:105270003EBD1F203EBDDFF8780400F024FA212057
:105280003EBD00BF25377800DFF8680400F01BFA48
:1052900021203EBD0FF2E841E06A00F0CFFA00F0B5
:1052A0002EFB01203EBD00003D0D0000DFF8340460
:1052B0000022DFF84434C0E90423DFF83014C1E9E8
:1052C0000423DFF83824DFF83834C0E90623C1E9C5
:1052D0000623DFF83034C0E90823C1E9082301229E
:1052E00002731046087300F0D9BA00002533780025
:1052F00010B582B003E0DFF81034FCF7ABFA0022FF
:105300001346FBF7BBFFF6D3DFF8D843D4E90423F9
:10531000FCF74EF8FCF774FA2060C0F307410091E7
:10532000C0F30723C2B20FF26041E06A00F086FAD0
:10533000BDE8134000F0E3BA10B582B003E0DFF837
:10534000C833FCF787FA00221346FBF797FFF6D322
:10535000DFF89843D4E90423FCF72AF8FCF750FA65
:105360002060C0F307410091C0F30723C2B20FF2DF
:105370001841DC48C06A00F061FABDE8134000F053
:10538000BEBA10B5D74C0120E0736068FCF7FAF89C
:10539000D4E90423FCF704F92268B2F1807F01D933
:1053A00081F00041227B002A06D0022A02D181F03E
:1053B000004110BD0020014610BD10B5CB4C0120AE
:1053C000E0736068FCF7DEF8D4E90423FCF7E8F842
:1053D0002268B2F1807F01D981F00041227B002A4E
:1053E00006D0022A02D181F0004110BD0020014602
:1053F00010BDBC48017B022901D103210173017B4F
:10540000002901D1012101730021C1817047B748F2
:10541000017B022901D103210173017B002901D104
:10542000012101730021C181704710B5AD4C206886
:10543000FCF7A8F8D4E90423BDE81040FCF7B0B8A5
:1054400010B5AA4C2068FCF79DF8D4E90423BDE808
:105450001040FCF7A5B810B5A24CA27B002A39D0A9
:105460000122E273227B012A06D0032A0FD0052AEB
:1054700019D0072A22D010BDA068FCF783F8024695
:105480000B46D4E90601BDE81040FCF789B8A068D6
:10549000FCF778F802460B46D4E90601FCF780F8E1
:1054A00081F0004110BDA068FCF76CF802460B4685
:1054B000D4E90801BDE81040FCF772B8A068FCF719
:1054C00061F802460B46D4E90801FCF769F881F05F
:1054D000004110BD0020014610BD10B5834CA27BD9
:1054E000002A39D00122E273227B012A06D0032A46
:1054F0000FD0052A19D0072A22D010BDA068FCF7CA
:1055000041F802460B46D4E90601BDE81040FCF71D
:1055100047B8A068FCF736F802460B46D4E9060106
:10552000FCF73EF881F0004110BDA068FCF72AF8B6
:1055300002460B46D4E90801BDE81040FCF730B83C
:10554000A068FCF71FF802460B46D4E90801FCF7F7
:1055500027F881F0004110BD0020014610BD30B594
:10556000A3B06A4AD1E91045CDE92045D1E90E45FD
:10557000CDE91E45D1E90C45CDE91C45D1E90A45E7
:10558000CDE91A45D0E91045CDE91845D0E90E45D9
:10559000CDE91645D0E90C45CDE91445D0E90A45D9
:1055A000CDE91245D1E90845CDE91045B1F91A30E8
:1055B0000F93B1F918300E93D1E90445CDE90C45AC
:1055C000D1E90245CDE90A45B1F90010895C08919D
:1055D000D0E90845CDE90645B0F91A100591B0F9B2
:1055E00018100491D0E90445CDE90245D0E90245FF
:1055F000CDE90045B0F90000825C0FF29C113948FA
:10560000C06A00F01BF923B0BDE8304000F077B964
:1056100030B593B005460C4604F14000119004F1FA
:105620003800109004F130000F9004F128000E9023
:1056300005F140000D9005F138000C9005F13000A7
:105640000B9005F128000A9004F12000099004F164
:105650001A00089004F11800079004F11000069059
:1056600004F10800059012A8049005F120000390B1
:1056700005F11A00029005F11800019005F11000E3
:10568000009005F108030DF14A020FF26411204861
:1056900000F0B0F99DF84A002D2801D1012000E06A
:1056A000002028809DF848002D2801D1012000E02D
:1056B0000020208009A10B48C06A00F0BFF800F06C
:1056C0001EF913B030BD80B5024605A10548C06A79
:1056D00000F0B4F8BDE8014000F011B93D0D000044
:1056E00025730000101100204411002070130020C9
:1056F0007C480008A4480008807AD840FB0811358F
:10570000BB36C240BB360241008076400C110020FF
:10571000471100203D3030423238390D0000000082
:105720003D21310D000000003D4137464430300D31
:10573000000000003D3030443830300D00000000E3
:105740003D3032303330310D000000003D257825EA
:105750007825780D000000003D31300D000000007C
:105760003D3143303530310D000000003D36D13041
:105770003230300D000000003D21330D00000000EC
:105780003D21300D000000003D25303258253032DB
:1057900058253032580D0000256320252E31662013
:1057A000256C6620256420256420252E3266202560
:1057B0006320252E316620256C6620256420256413
:1057C00020252E326620252E326620252E32662098
:1057D000252E326620252E326620252E3266202583
:1057E0002E326620252E326620252E32660D0000D0
:1057F00025317320256C6620256C662025642025C4
:105800006420256C662025317320256C6620256C6C
:105810006620256420256420256C6620256C662082
:10582000256C6620256C6620256C6620256C66201C
:10583000256C6620256C6620256C66000CB41CB5B2
:10584000044604A801900A46009401AB00A9074849
:1058500078441830FCF79AFF009A00211170002854
:105860005CBF0098001B16BC5DF80CFB8BBFFFFFF4
:10587000012100F01F029140524A400942F82010D5
:1058800070470901002806D54F4A00F00F00801824
:1058900000F8041C70474D4A8154704780B500F0F1
:1058A000C8F84B48016841F4804141F001010160B2
:1058B0004848016841F030010160016821F0C001F1
:1058C0000160016841F0800101604348818841F036
:1058D0000C0181804FF41C610180018841F00401BA
:1058E0000180818841F4005141F0600181800F21E5
:1058F0002520FFF7C6FF2520BDE80240B8E737485E
:1059000041780029FDD136490978364A118041781D
:10591000491C41707047F0B5334E3788B6F804C063
:1059200007F02700202836D13048D0E9004542F260
:105930001070002120186941DFF8B4E0DEE934235B
:105940009D4208DB01DC944205D3CEE934010020FE
:105950008EF8000001E0CEE934019EF80000002836
:1059600006D1BCF13A0F16D101208EF8000012E0EA
:1059700000EB0E0181F804C0401C8EF80000BCF161
:105980000D0F08D1801E8EF8040000208EF8000054
:10599000012012490870780611D510481049427844
:1059A000515C002904D0B1804178491C417001E06C
:1059B0000021417030884FF6BF7108403080F0BD43
:1059C0000000000000E100E018ED00E000E400E06D
:1059D0001810024004080140083801403814002023
:1059E0001812002004380140003801403014002013
:1059F000401100200DB400B582B004A800900A4602
:105A000000AB03A9034878440A30FDF799FD06BCB2
:105A10005DF810FB3FBBFFFF0901002806D5374AA0
:105A200000F00F00801800F8041C7047344A8154BD
:105A3000704710B5334C45F6C0506060206840F0A8
:105A4000040020600020A060206840F00100206079
:105A500001214FF0FF30FFF7DFFF206840F0020028
:105A6000206010BD2848D0E90023521C43F10003F8
:105A7000C0E90023704730B40299002818D02248AA
:105A80000C78002C07D101240C70D0E90045A21835
:105A90006B41C1E90223D0E90023D1E90245AB42C1
:105AA00008DB01DCA24205D300200870012002E0DF
:105AB00000200870002030BC704730B402990028E4
:105AC00016D011480C78002C07D101240C70D0E9B5
:105AD0000045A2186B41C1E90223D0E90023D1E9B6
:105AE0000245AB4206DB01DCA24203D3012002E007
:105AF00000200870002030BC7047000018ED00E066
:105B000000E400E010E000E030140020000000009D
:105B100010B4794B0468A24203D36F20187002209E
:105B20000AE01A7851180068814203D36F20187078
:105B3000012001E00020187010BC70471CB501E086
:105B4000FBF76CFB4FF4D06240F63B016B48FFF76C
:105B5000DFFF002803D0022816D005D322E04FF043
:105B60008040674948601DE0664800904FF47A72B3
:105B700000230120FFF77FFF002813D06048016851
:105B800081F4804101600DE05E48009064220023B2
:105B90000120FFF770FF002804D05948016881F404
:105BA0008041016058499DF80400002809D05448FC
:105BB000026882F40052026000208DF80400087030
:105BC0000CE000914FF47A7200230120FFF775FF7B
:105BD000002803D04FF400504949486001A8FFF75E
:105BE00097F8C01E1D28ADD8DFE800F011180F107F
:105BF00010101010202A343E101010101010252FF5
:105C00003943101010101010534899E79AE7FBF72A
:105C1000F2FA002896D1FFF7ECFB93E7FBF7F6FAD0
:105C200000287FF48FAFFFF7F2FB8BE7FBF76AF9F1
:105C3000FFF75EFB86E7FBF77DF9FFF77DFB81E76A
:105C4000FFF7F3FBFBF73EF87CE7FFF7F9FBFBF709
:105C50004CF877E7FFF7FFFBFBF75EF872E7FFF71B
:105C60003CFCFBF7DBF86DE7FFF78BFBFBF77CF900
:105C700068E7FFF7A2FBFBF725FA63E7234C24490B
:105C80002046FFF7C5FC90222146224800F0C8F8C4
:105C900013BD1F491D48FFF762FC53E738B500F0FC
:105CA000F5F800F031F9FBF711FB4FF400501A49F9
:105CB0000860184C154D90222946204600F095F8B2
:105CC000B5F91A0000280FD128460FF254014822D6
:105CD000FDF7C4FB0E4829464822FDF7BFFB902282
:105CE0002946204600F09CF8FFF7E0FAFAF7B1FBEE
:105CF000FFF724FFDFE700003A1400203C240140B6
:105D00000C100140C8130020B8130020E01200203E
:105D10002813002000FC01081010014000000000C2
:105D20000000000000000000000000000000F03F44
:105D300000000000000886402003C80000000000AA
:105D4000000000000000E03F000000000000F03F05
:105D50000000000000000000000000000000000043
:105D600000000000000000004248006800F0010050
:105D700080F00100704710B500F016F83E4C206826
:105D800040F0020020603D486060206840F0400024
:105D90002060FFF7E9FF0028FBD0206820F0020018
:105DA0002060BDE8104005E03548364901603649BD
:105DB000016070473048016841F080010160704720
:105DC00038B504460D46FFF7CFFF0028FBD02580ED
:105DD000FFF7CAFF0028FBD0280C6080FFF7C4FF44
:105DE0000028FBD031BD0068704770B582B0044612
:105DF0000D46164606E0241D2046FFF7F4FF45F841
:105E0000040B361F042EF6DA002E08D02046FFF7CA
:105E1000EAFF0090324600A92846FDF71FFB73BD3C
:105E2000F8B504460D461646FFF7A5FFFFF7BCFF81
:105E3000114F386840F00100386006E0241D55F825
:105E4000041B2046FFF7BCFF361F042EF6DA002E97
:105E500008D03246294600A8FDF700FB00992046ED
:105E6000FFF7AEFF3868400840003860FFF7A2FF38
:105E7000F1BD00000C2002401020024000FC01088F
:105E80000420024023016745AB89EFCD57480168E4
:105E90008907FCD5016841F48031016001688903FC
:105EA000FCD541684160416841604168416041689A
:105EB00021F47C114160416841F400314160416846
:105EC00041F480314160416841F4801141600168D2
:105ED00041F08071016001688901FCD54168890841
:105EE00089004160416841F002014160416801F070
:105EF0000C010829FAD1816941F0040181618169AD
:105F000041F008018161704730B43948016841F0BF
:105F100004010160016841F008010160016841F07D
:105F200010010160016841F00101016031490A6816
:105F300042F000720A6030494A6842F440124A60F6
:105F40004A6822F440024A604A6842F040724A605D
:105F50004A6822F040624A60284A136843F04C5372
:105F6000136013686FF0434423401360244B1C6894
:105F700044F033041C601C6824F0CC041C605C6892
:105F8000204D2C435C605C681F4D2C405C601368A6
:105F900023F0CC0313600A6822F033020A60016820
:105FA00041F4007101601948016841F4A061016089
:105FB0004168174A11434160416B41F02001416340
:105FC000416B41F480414163416B41F400214163E5
:105FD000416B41F440114163416841F0010141606E
:105FE000416841F40011416030BC7047001002402C
:105FF0001810024004000140001001400008014058
:10600000000C014000003033FFFF3F330424014007
:1060100002F08000816807E00268116853688918FF
:106020005B18C36008320260C2689142F4D04A1C17
:1060300082600878704738B504460D46A068E1686C
:10604000884212D120686168884208BF00F0C3F816
:106050002068227C016802B14944A160426852185C
:10606000E260083091422060ECD0A068401CA06043
:1060700000F8015D31BD2DE9F0418AB000F1080161
:1060800005910268520801EBC201069100210791B7
:1060900008910168490800EBC101083100910179BC
:1060A00001F001018DF8101040680099400801EBE3
:1060B000C000019000200290039084E005A8FFF743
:1060C000A9FF044614F0030603D105A8FFF7A2FFB9
:1060D000C61C25090F2D1BD105A8FFF79BFF00F15A
:1060E0000F0515E00598016808180599079049689B
:1060F0000818089005980830059007980899884274
:10610000F0D0401C079010F8011D00A8FFF793FF86
:10611000761EF2D1002D51D005A8FFF77BFF064671
:10612000A00800F00300032804BF05A8FFF772FFD2
:10613000DDF800800299039F06EB002008E0A8F13B
:106140000808A8F10801801A0A6849688F183946BA
:1061500058F8082C8A1A8242F1D30C1AAE1C2DD0A2
:10616000BC4206D158F8044B58F8040B0719BC423E
:10617000F8D00298039914F8015B884217D100986F
:106180000199884208BF00F026F8009800689DF841
:106190001010029009B14844029000990298496891
:1061A000009A09180832884203910092E7D00298B9
:1061B000401C0290761E00F8015DD1D1029803992F
:1061C00088427FF47BAF0198009981427FF476AFDB
:1061D0000AB0BDE8F081012000F000B880B5C046EB
:1061E000C046024A11001820ABBEFBE726000200A1
:1061F0000D48016841F00101016041680B4A1140FE
:10620000416001680A4A11400160016821F480215F
:106210000160416821F4FE0141604FF41F0181607B
:106220000021C16206E00000001002400000FFF8FB
:10623000FFFFF6FE7047000010B50749794418319A
:10624000064C7C44163404E00A68081D511888473F
:106250000146A142F8D110BD080000003000000046
:106260004BB0FFFFFC0200004011002000000000C6
:1062700007FEFFFF020000000200000024010000F2
:1062800032080000000000204011000000F00BF870
:10629000002801D0FFF7D0FF0020C046C046FFF71E
:1062A000FDFC00F002F80120704700F001B800008A
:1062B00007463846FFF792FFFBE70000014880479A
:1062C00001480047F1610008CD620008C046C046A1
:1062D000C046C046FFF7DAFFFFF7FEBFFFF7FEBF7D
:1062E000FFF7FEBFFFF7FEBFFFF7FEBFFFF7FEBFE2
:1062F000FFF7FEBFFFF7FEBFFFF7B4BBFFF7FEBF20
:10630000FFF7FEBFFFF7FEBFFFF7FEBFFFF7FEBFC1
:10631000FFF7FEBFFFF7FEBFFFF7FEBFFFF7FEBFB1
:10632000FFF7FEBFFFF7FEBFFFF7FEBFFFF7FEBFA1
:10633000FFF7FEBFFFF7FEBFFFF7FEBFFFF7FEBF91
:10634000FFF7FEBFFFF7FEBFFFF7FEBFFFF7FEBF81
:10635000FFF7FEBFFFF7FEBFFFF7FEBFFFF7FEBF71
:10636000F9F7FEBEFFF7FEBFFFF7FEBFFFF7FEBF68
:10637000FFF7FEBFFFF7FEBFFBF7D1BDFFF7FEBF84
:10638000FFF7C9BAFFF7FEBFFFF7FEBFFFF7FEBF7B
:10639000FFF7FEBFFFF7FEBFFFF7FEBFFFF7FEBF31
:1063A00000FE64002D01F601BF02880351041A05A6
:1063B000E305AC0675073D080609CE09970A5F0B91
:1063C000270CEF0CB70D7F0E470F0E10D6109D1146
:1063D00064122B13F213B8147F1545160A17D01741
:1063E00096185B19201AE41AA91B6D1C311DF51DA6
:1063F000B81E7B1F3E200021C22184224523072492
:10640000C724882548260727C72786284429022A23
:10641000C02A7D2B3A2CF72CB32D6E2E292FE42F7A
:106420009E3058311132CA3282333A34F234A835B0
:106430005F361437CA377E383239E639993A4C3BE1
:10644000FD3BAF3C603D103EBF3E6E3F1D40CA402D
:1064500077412442D0427B432544CF4478452146AE
:10646000C94670471648BC486149064AA94A4C4B80
:10647000EF4B904C314DD14D704E0F4FAC4F4950BA
:10648000E55081511C52B5524E53E7537E54155579
:10649000AB554056D4566757F9578B581C59AC59D1
:1064A0003B5A10FDC95A565BE35B6E5CF95C835D39
:1064B0000B5E935E1A5FA05F2660AA602D61B061DB
:1064C0003162B2623163B0632D64AA642665A0654F
:1064D0001A6693660B678267F7676C68E0685369B2
:1064E000C469356AA56A136B816BEE6B596CC46C19
:1064F0002D6D966DFD6D636EC96E2D6F906FF26F91
:106500005370B37012716F71CC7127728272DB722B
:1065100033738A73E07335748974DB742D757D75FC
:10652000CC751B766876B376FE7647779077D7770B
:106530001D786278A678E8782A796A79A979E77966
:10654000247A5F7A9A7AD37A0B7B427B777BAC7B17
:10655000DF7B117C427C717CA07CCD7CF97C247D2E
:106560004E7D767D9D7DC37DE87D0C7E2E7E4F7EAB
:106570006F7E8E7EAB7EC87EE37EFD7E157F2D7F97
:10658000437F587F6B7F7E7F8F7F9F7FAE7FBC7FF7
:10659000C87FD37FDD7FE57FED7FF37FF87FFC7FD2
:1065A000FE7FFF0212FE0A12F81212ED1A12DD220D
:1065B00012C82A12AE32128F3A126B4212434A109C
:1065C00001157FFD5612C85E128E66124F6E1001C5
:1065D0000C7EE87A129D8210034E7D247DF9921282
:1065E000A09A1003427C117CDFAA1277B210010B33
:1065F0007BD3BE10035F7A247AE7CE10036A792A30
:1066000079E8DE100362781D78D7EE10014777FE37
:10661000FA140368761B76CC0A14012D75DB161468
:10662000013574E02214013373DB2E14012772CC80
:106630003A14051271B3705370F24E14052D6FC9E0
:106640006E636EFD6214052D6DC46C596CEE76148C
:106650000D136BA56A356AC4695369E0686C68F705
:106660009A14100B6793661A66A0652665AA642DB6
:1066700064B0633163C200FE62B0612D61AA60261E
:1066800060A05F1A5F935E0B5E835DF95C6E5CE3F6
:106690005B565BC95A3B5AAC591C598B58F9576722
:1066A00057D4564056AB5515557E54E7534E53B507
:1066B000521C528151E5504950AC4F0F4F704ED192
:1066C0004D314D904CEF4B4C4BA94A064A6149BCA9
:1066D0004816487047C94621467845CF4425447B33
:1066E00043D04224427741CA401D406E3FBF3E1016
:1066F0003E603DAF3CFD3B4C3B993AE63932397E3A
:1067000038CA3714375F36A835F2343A348233CA80
:1067100032113258319E30E42F292F6E2EB32DF7CF
:106720002C3A2C7D2BC02A022A44298628C7270709
:106730002748268825C724072445238422C2210010
:10674000213E207B1FB81EF51D311D6D1CA91BE4C9
:106750001A201A5B199618D0170A1745167F15B814
:1067600014F2132B1364129D11D6100E10470F7FD5
:106770000EB70DEF0C270C5F00FE0B970ACE090633
:10678000093D087507AC06E3051A0551048803BFE7
:1067900002F6012D0164009CFFD3FE0AFE41FD7844
:1067A000FCAFFBE6FA1DFA54F98BF8C3F7FAF632A0
:1067B000F669F5A1F4D9F311F349F281F1B9F0F2D8
:1067C000EF2AEF63EE9CEDD5EC0EEC48EB81EABBD3
:1067D000E9F6E830E86AE7A5E6E0E51CE557E4936A
:1067E000E3CFE20BE248E185E0C2DF00DF3EDE7C82
:1067F000DDBBDCF9DB39DB78DAB8D9F9D839D87AFE
:10680000D7BCD6FED540D583D4C6D309D34DD292BA
:10681000D1D7D01CD062CFA8CEEFCD36CD7ECCC69E
:10682000CB0ECB58CAA1C9ECC836C882C7CEC61A8F
:10683000C667C5B4C403C451C3A0C2F0C141C1926C
:10684000C0E3BF36BF89BEDCBD30BD85BCDBBB311C
:10685000BB88BADFB937B990B8EAB744B79FB6FA80
:10686000B557B5B4B411B470B3CFB22FB290B1F183
:10687000B054B0B7AF1BAF7FAEE400FEAD4BADB2CE
:10688000AC19AC82ABEBAA55AAC0A92CA999A80750
:10689000A875A7E4A654A6C5A537A5AAA41DA492C9
:1068A000A307A37DA2F5A16DA1E6A060A0DA9F5683
:1068B0009FD39E509ECF9D4E9DCF9C509CD39B5668
:1068C0009BDA9A609AE6996D99F5987E9809989462
:1068D000972097AD963C96CB955B95ED947F94125F
:1068E00094A7933C93D3926A9203929D913791D34C
:1068F0009070900E90AD8F4D8FEE8E918E348ED91C
:106900008D7E8D258DCD8C768C208CCB8B778B25B9
:106910008BD38A838A348AE58998894D890289B91B
:106920008870882988E3879E875A871887D6869635
:106930008657861986DC85A18566852D85F584BEFA
:1069400084898454842184EF83BE838F836083335E
:10695000830783DC82B2828A8263823D821882F45A
:1069600081D281B18191817281558138811D8103EC
:1069700081EB80D380BD80A880958082101A8071C1
:106980008061805280448038802D8023801B80135A
:10699000800D80088004800280010212020A120821
:1069A0001212131A12232212382A12523212713A78
:1069B00012954212BD4A1001EB80035612385E1246
:1069C000726612B16E1001F481187A12638210039C
:1069D000B282DC82079212609A1003BE83EF832199
:1069E000AA1289B21001F5842DBE1003A185DC85A1
:1069F00019CE10039686D68618DE10039E87E3878D
:106A000029EE1001B98802FA14039889E589340A3D
:106A10001401D38A25161401CB8B20221401CD8CAE
:106A2000252E1401D98D343A1405EE8E4D8FAD8F7D
:106A30000E4E1405D39037919D9103621405D392A5
:106A40003C93A7931276140DED945B95CB953C96F1
:106A5000AD9620979497099A1410F5986D99E69938
:106A6000609ADA9A569BD39B509CCF9CC200FE9DA5
:106A7000509ED39E569FDA9F60A0E6A06DA1F5A11F
:106A80007DA207A392A31DA4AAA437A5C5A554A6B9
:106A9000E4A675A707A899A82CA9C0A955AAEBAA8E
:106AA00082AB19ACB2AC4BADE4AD7FAE1BAFB7AFB0
:106AB00054B0F1B090B12FB2CFB270B311B4B4B43E
:106AC00057B5FAB59FB644B7EAB790B837B9DFB94A
:106AD00088BA31BBDBBB85BC30BDDCBD89BE36BFEF
:106AE000E3BF92C041C1F0C1A0C251C303C4B4C44A
:106AF00067C51AC6CEC682C736C8ECC8A1C958CA6F
:106B00000ECBC6CB7ECC36CDEFCDA8CE62CF1CD07F
:106B1000D7D092D14DD209D3C6D383D440D5FED598
:106B2000BCD67AD739D8F9D8B8D978DA39DBF9DBD5
:106B3000BBDC7CDD3EDE00DFC2DF85E048E10BE24E
:106B4000CFE293E357E41CE5E0E5A5E66AE730E829
:106B5000F6E8BBE981EA48EB0EECD5EC9CED63EE80
:106B60002AEFF2EFB9F081F149F211F3D9F3A1FC68
:106B70001BFFF469F532F6FAF6C3F78BF854F91DEA
:106B8000FAE6FAAFFB78FC41FD0AFED3FE9CFF005B
:106B900006FDFF0006FDFF0006FDFF0006FDFF00ED
:106BA00006FD9F0006FDFF000EFDDF000EF2560001
:106BB0000113ABAA01F0011C7AF84235F0015B40E9
:106BC000CF4080F3192B2D500006381400201812E6
:026BD0000020A3
:04000005080062CDC0
:00000001FF
